:020000040000FA
:1000000021EF02F01200FFFF04EF04F01200FFFFE7
:100010000600FFFFFFFFFFFF0CEF04F01200FFFFE1
:10002000F26AD19001EC02F0BFEC01F0ECEF00F0CD
:10003000120000001200F1EC01F0F1EC01F0F1EC23
:1000400001F0F1EC01F0F1EF01F0900E006ED00E36
:10005000016E030E026E036A9EAA2BD0D7EC01F04C
:10006000000927E009503B0A21E0790A02E0046A0E
:1000700020D0C10E8A16042A030E045C04E335EC7A
:1000800001F0010E22D00450010A0DE0030A09E03C
:10009000010A05E0070A01E008D08A8406D08A86B2
:1000A00004D08A8802D08A8A00D003D03B0EAD6E7D
:1000B00000D00006000E015A025A035A00500110E7
:1000C00002100310C9E1000E00D0120001EC02F092
:1000D000B2DFBFEC01F0B9DF000911E1000EF66EEE
:1000E000080EF76E0900F5CF0EF00800F5CF0FF0FF
:1000F0000E500F1007E06FEC01F0000903E1ECEF88
:1001000000F004D08A90919601EF04F01200ECEC1C
:1001100001F0052A000E062205A802D0918601D022
:1001200091961200ECEC01F0052A000E062206AAB8
:1001300002D08A8001D08A901200610EE96E000E12
:10014000EA6EA5EF01F0FF00120092EC00F09EAA0B
:1001500012D0D7EC01F000090EE0490E095C03E073
:10016000420E095C02E181D806D00950AD6E440E02
:10017000095C01E101D0E9D712000001E1510E6EE6
:100180000F6A0E507F0B02E0000E08D0E1C0F6FFB0
:10019000E2C0F7FFE3C0F8FF010E00D01200F46ADE
:1001A000610EE96E000EEA6E9EAAFED7D7EC01F052
:1001B000000902E1000E0FD00950EF6EEE50F42658
:1001C000E50EE95C000EEA58EFE3F45002E1010E9F
:1001D00002D0000E00D012000001606B9196B5DFD6
:1001E0008A90056A066ADBDF000903E14E0EAD6EF8
:1001F00035D0C3DF000903E14E0EAD6E2FD0020EE5
:10020000F85C0BE1F66A080EF76EF86A6BEC01F029
:1002100094DF420EAD6E23D021D0000EF65C080EA6
:10022000F758000EF85803E2410EAD6E17D0800E5D
:10023000F65CFD0EF758010EF85803E34E0EAD6E56
:100240000DD00001605105E1010E606F59EC01F025
:1002500094DF73DF410EAD6E87EC00F0C4D7ACA223
:10026000FED7ECEC01F0A3EF00F06B0EE66ECAECEB
:1002700001F0E552780EE66ECAEC01F0E552700E20
:10028000E66ECAEC01F0E552610EE66ECAEC01F0D2
:10029000E552310EE66ECAEC01F0E552300EE66E24
:1002A000CAEC01F0E552300EE66ECAEC01F0E55200
:1002B0001200F66A080EF76EF86A0DD8800EF62660
:1002C000000EF722F822800EF65CFD0EF758010EA4
:1002D000F858F3E31200940E7F6E9DEF01F0076A69
:1002E000086AF66A080EF76EF86A0900F550F46EAF
:1002F0000900F550F36EF3500726F450082207501A
:10030000081002E1010E18D00900F550F46E090042
:10031000F550F36EF3500726F4500822800EF65C79
:10032000FD0EF758010EF858EFE30750081002E1F0
:10033000010E02D0000E00D01200550E7E6EAA0EE5
:100340007E6E7F8200007F941200010EF46E0A0020
:10035000800EF36EEE50F56E0F00F306F3500008BA
:10036000F9E3840E7F6EE9DFF406F4500008F0E351
:1003700012009EAA03D0AE50E86EFBD71200040E06
:10038000AC6E100EAB6E656A190EAF6EAC8AAB8E9A
:10039000B9EF01F0D9CFE6FFE1CFD9FFACA2FED78C
:1003A000FE0EDB50AD6EE552E7CFD9FF12009EAADC
:1003B00010D0ABA204D0AB98AB88DBDF09D0ABA4E4
:1003C00003D0AE50E86E04D0AE50096E010E03D0DB
:1003D000EED7000E00D01200140E0A6E0B6AF7EF73
:1003E00001F0200E0A6E4E0E0B6EF7EF01F00A06BA
:1003F000000E0B5A0A500B1003E000000000F7D764
:1004000012000F015F0E256F020E246F400E236F46
:100410008A6A8B6A8C6E100E8D6E8E6A8F6A300EB1
:10042000906E916A3F0E926E936AB80E946E956AC2
:10043000966A120E976E240E986E220E996E9A6A24
:1004400012001EEE00F02EEE00F0F86A0D9C80EC1B
:1004500002F031EC02F01AEC00F066EC00F0FBD791
:100460001200320EF66E000EF76E000EF86E0F01DF
:100470000900F550056F0900F550066F03E10567A7
:1004800001D03DD00900F550006F0900F550016F13
:100490000900F550026F09000900F550E96E0900E6
:1004A000F550EA6E090009000900F550036F0900D4
:1004B000F550046F09000900F6CF07FFF7CF08FFDA
:1004C000F8CF09FF00CFF6FF01CFF7FF02CFF8FF0B
:1004D0000F01035302E1045307E00900F550EE6EEB
:1004E0000307F8E20407F9D707CFF6FF08CFF7FFB5
:1004F00009CFF8FF0F010507000E065BBFD71200FA
:10050000160EF36E00EE00F00F0E01D81200EA6036
:1005100002D0EE6AFCD7F350E9601200EE6AFCD715
:10052000FFFFFFFFFFFFFFFFFFFFFFFFFFFFFFFFDB
:10053000FFFFFFFFFFFFFFFFFFFFFFFFFFFFFFFFCB
:10054000FFFFFFFFFFFFFFFFFFFFFFFFFFFFFFFFBB
:10055000FFFFFFFFFFFFFFFFFFFFFFFFFFFFFFFFAB
:020800000000F6
:0608020035EF4CF012007E
:040808000BEF31F0D1
:040818001AEF3CF0A7
:1008200007004C9900003A070000060000004B99B1
:10083000000069070000010000004A9900006807F5
:10084000000001000000479900005B070000030062
:1008500000001099000080060000370000000C998D
:1008600000004E0700000400000095970000670795
:0608700000000100000081
:0A0876003FEC0CF006E142EC0CF040
:1008800069C7E6FF20EC0DF095EF0BF07AEC0CF069
:10089000410847E149EC0CF012E18BEC0CF0DF6A07
:1008A0000B0EDF5C09E0DFCFE6FF66EC1AF0E552E5
:1008B000C5EC0BF0DF2AF4D79EEC0BF04BD064ECC8
:1008C0000CF011E1040EFDEC0BF044E3040E7CECA3
:1008D0000BF033083FE3DF6A0B0EDF5C3BE0040EF6
:1008E000C2EC0CF0F9D70F0EE3EC0CF033E1DF6A49
:1008F0000B0EDF5C0DE0040EDF24FDEC0BF02AE3B1
:10090000040EDF247CEC0BF0330824E3DF2AF0D75D
:10091000DF6A0B0EDF5C1EE0040EDF24C2EC0CF07D
:10092000F8D759EC0CF016E064EC0CF00AE1D7ECC7
:100930000CF066EC1AF0E552C5EC0BF0E0EC0CF0B4
:1009400008D0AAEC0CF006E1050E7CEC0BF00CECE8
:100950000CF0E552E55295EF0BF02EEC0DF0320A5B
:100960001AE0030A15E0010A0BE00B0A1DE176EC20
:1009700047F0F2EC0CF087EC47F0E552E55214D06A
:100980000001010EFC6F76EC47F0010807E103D08F
:100990000001010E02D00001020EFC6F49EC0CF0C8
:1009A00003E10001FA81FA8595EF0BF082EC0CF07F
:1009B000030EE3EC0CF009E106012551E66EE66A50
:1009C0008FEC0BF06FEC0BF016D0C7EC0CF015E0D1
:1009D000AAEC0CF012E173EC0CF0010EDB500DE10F
:1009E000DFCF25F6010EE66E250EE66E060EE66EEC
:1009F000250E08EC0CF0BDEC0BF0020EE15C02E2FF
:100A0000E16AE552E16E95EF0BF077EC0CF010E047
:100A1000010A08E00B0A11E145EC0CF065EC41F02D
:100A2000E5520BD049EC0CF008E10DEC41F005D09B
:100A300049EC0CF002E14CEC41F095EF0BF00DECC1
:100A40000DF029E0050E7CEC0BF0310A16E0010AEE
:100A50000CE00B0A20E1D7EC0CF073EC1AF0E55235
:100A6000C5EC0BF0E0EC0CF015D0AAEC0CF013E1A7
:100A700007014CA710D0E66A08D0AAEC0CF00BE1F5
:100A800007014CA708D0010EE66EDFCFE6FFA1EC10
:100A90001BF0E552E552E55295EF0BF01DEC0DF021
:100AA000E126ECEC0BF07FEC0BF0D4EC0BF025E046
:100AB00064EC0CF00EE1D7EC0CF0B5EC1AF0E5525A
:100AC000F2EC0CF0A5EC34F0E552E552E0EC0CF061
:100AD00013D0ADEC0CF011E1050E97EC0CF018EC16
:100AE0000CF0020EDB5009E1010EDBCFE6FFDFCF99
:100AF000E6FFC5EC1BF0E552E552030EE15C02E2B5
:100B0000E16AE552E16E95EF0BF01DEC0DF0E12688
:100B1000E3EC0CF007E136C7E6FF45EC0CF0F5EC32
:100B20001FF024D059EC0CF023E064EC0CF020E131
:100B300007013651DF5C1CE0DFCFE6FF85EC1AF0E1
:100B400018EC0CF020500EE020EC0CF0DFCFE6FFAC
:100B5000E66A2F0EE66EE66A1CEC2DF0146E060EA9
:100B6000E15E145020EC0CF049EC0BF0E552E5523C
:100B7000030EE15C02E2E16AE552E16E95EF0BF0F3
:100B80007AEC0CF0580A05E0080A56E127C6DFFFA8
:100B900002D028C6DFFF49EC0CF017E18BEC0CF01B
:100BA000DF50CF0A0CE0A80A08E0540A04E02A0A41
:100BB00009E1330E05D0320E03D0310E01D0300ED4
:100BC00092EC0BF09EEC0BF037D064EC0CF034E1BF
:100BD000040E7CEC0BF0330A0CE0010A08E0030A77
:100BE00004E0010A29E1CF0E05D0670E03D0330ED1
:100BF00001D0190EDF6E40EC0BF031EC0DF0500817
:100C00000EE1DFCF27F6010EE66E270EE66E060E2A
:100C1000E66E270EBBEC0CF0E1EC37F00DD0DFCF29
:100C200028F6010EE66E280EE66E060EE66E280E1B
:100C3000BBEC0CF002EC38F0E55295EF0BF07AECDF
:100C40000CF04E0A1CE0750A04E064EC0CF01FE0A6
:100C500030D042EC0CF007014CA307D078EC40F008
:100C6000F2EC0CF098EC34F005D04E0EF2EC0CF0F7
:100C700023EC38F0E552E552E0EC0CF019D049ECE9
:100C80000CF017E107014C9336C7E6FF0FD0ECECF0
:100C90000BF0030E7FEC0BF0B7EC35F0E552DAEC1D
:100CA0000CF007E007014C83DFCFE6FFDAEC40F001
:100CB000E552E55295EF0BF02EEC0DF04E0A10E0E8
:100CC0000C0A08E0790A11E145EC0CF0EBEC47F076
:100CD000E5520BD049EC0CF008E10501E29F05D08C
:100CE00049EC0CF002E10501E28F95EF0BF03FECCF
:100CF0000CF007E131EC43F0F2EC0CF046EC43F081
:100D00000CD064EC0CF00BE1D6EC28F0000907E104
:100D1000E30EE66E050E9CEC0CF0E552E55295EF05
:100D20000BF077EC0CF010E0010A08E00B0A11E17F
:100D300019EC0DF0010BB0EC0CF00BD049EC0CF001
:100D400008E107014C9105D049EC0CF002E10701E4
:100D50004C8195EF0BF00DEC0DF01DE064EC0CF008
:100D600009E142EC0CF0CAEC0CF0D4EC1AF028ECDF
:100D70000DF010D0BEEC0CF00EE0090EE3EC0CF020
:100D80000AE1050EA1EC0BF0DFCFE6FFF9EC1BF05A
:100D9000E552E552E552E55295EF0BF099EC0BF078
:100DA000050E61EC0CF00EE0ADEC0CF00BE142EC4A
:100DB0000CF0030EA1EC0BF045EC0CF065EC17F019
:100DC0005EEC0CF095EF0BF00DEC0DF01DE064EC1B
:100DD0000CF009E142EC0CF0CAEC0CF0C1EC1AF09A
:100DE00028EC0DF010D0BEEC0CF00EE0090EE3EC98
:100DF0000CF00AE1050EA1EC0BF0DFCFE6FFDDEC15
:100E00001BF0E552E552E552E55295EF0BF03FEC51
:100E10000CF01BE182AA19D007014BB316D0F9ECF4
:100E20003DF08EEC3DF0DFEC19F0E66A0F0EE66E59
:100E300002EC15F0E552E55207014CA704D03CEC5A
:100E400044F006EC33F03AEC0BF095EF0BF077EC56
:100E50000CF012E0010A0AE00B0A13E119EC0DF0A4
:100E6000080B01E0010EB0EC0CF00BD049EC0CF0DB
:100E700008E107014C9705D049EC0CF002E10701AD
:100E80004C8795EF0BF0F5EC0CF00DE042EC0CF01C
:100E90008FEC0CF0490EFBEC0CF0C7C6E6FFC8C6A1
:100EA000E6FF01EC0DF0020EE15C02E2E16AE552C0
:100EB000E16E95EF0BF099EC0BF0E652AAEC0CF01A
:100EC00016E182AA14D007014BB311D0C7EC0CF085
:100ED0000EE059EC0CF00BE0050E7CEC0BF0030B74
:100EE000E66EDFCFE6FF02EC15F0E552E552E55283
:100EF00095EF0BF0F5EC0CF00BE042EC0CF08FEC06
:100F00000CF0500EFBEC0CF03AEC0CF001EC0DF098
:100F1000020EE15C02E2E16AE552E16E95EF0BF050
:100F200099EC0BF0E652FC0EDBCFE9FFDB2AFD0E5D
:100F3000DBCFEAFF01E3DB2AEFCFDFFFDF5009E081
:100F4000DFCFE6FF45EC0CF0B6EC0CF03B0EDF5CBF
:100F5000EAE1E552EAD3EDDB14CFE6FF15CFE6FF79
:100F600045EC0CF0B3EC4AF0EEEC0CF0DED33FECC9
:100F70000CF006E1FE0EDBCFFDF00001FA85FA8DE4
:100F8000D4D33FEC0CF006E145EC0CF013EC33F05D
:100F9000E55209D031EC0DF0430805E149EC0CF0C5
:100FA00002E1DEEC32F0C1D33FEC0CF007E104C605
:100FB000E6FF05C6E6FFB3DB9CDB14D007014CA7B8
:100FC00012D0030E97EC0CF0E552F3CF04F6F4CFF9
:100FD00005F6020EE66E040EE66E060EE66E040ED2
:100FE00008EC0CF0CADBA1D3A4DB07014CAB06D0A4
:100FF000FE0EDBCFFDF00001FA89FA8D96D33FECAF
:101000000CF006E1B7C6E6FFB8C6E6FF55EC0CF0FB
:101010008CD38FDB020EE3EC0CF004E0030EE3EC68
:101020000CF012E1D4DB490E7DDB4B0E7BDB580E5E
:1010300079DB500E77DB410E75DB310E73DB300E42
:1010400071DB300EDDEC0CF070D31ADB0FDBD190CE
:10105000F26A10EF00F0120077EC0CF012E0010AD7
:101060000AE00B0A13E119EC0DF0100B01E0010E80
:10107000B0EC0CF00BD049EC0CF008E107014C99F6
:1010800005D049EC0CF002E107014C894ED33FEC4E
:101090000CF007E1ABEC42F0F2EC0CF0C0EC42F0EB
:1010A0000CD064EC0CF00BE1D6EC28F0000907E161
:1010B000E40EE66E050E9CEC0CF0E552E55235D3DD
:1010C000DEDB04E1E2DBC2EC41F007D0E2DB06E16B
:1010D00031EC0DF0E66EDBEC41F0E55226D3CFDBD0
:1010E00005E114CFE6FF15CFE6FF08D0050EE9DBDA
:1010F00008E0ADEC0CF005E1030E23DBCADAE552A3
:10110000E55213D3F4DB18E0010A0DE00B0A23E1EA
:10111000B9DB07014BA502D0300E01D0310E02DB46
:10112000E0EC0CF017D0B5DB16E107014B8507ECBE
:1011300041F0205010E008D0ACDB0DE107014B95E9
:10114000205009E090B807D0D0EC0CF0E66A8ADABB
:10115000E552E552E552E9D292DB05E1CBC6E6FF66
:10116000CCC6E6FFA2DBE1D28ADB05E1D1C6E6FF11
:10117000D2C6E6FFC3DBD9D282DB0DE107014BA566
:1011800005D0DCC6E6FFDDC6E6FF04D0D8C6E6FF24
:10119000D9C6E6FFB3DBC9D272DB05E1DCC6E6FFE8
:1011A000DDC6E6FFABDBC1D2ADDB73DB60E131EC6A
:1011B0000DF04A0A40E0020A38E00F0A30E0010A66
:1011C00028E0030A20E0010A18E0070A10E0010AFB
:1011D00008E0030A4CE18050DF6E010E89CFDBFF8F
:1011E0002FD08150DF6E010E8ACFDBFF29D08250D5
:1011F000DF6E010E8BCFDBFF23D08350DF6E010E3D
:101200008CCFDBFF1DD08450DF6E010E8DCFDBFF56
:1012100017D08550DF6E010E8ECFDBFF11D08650C8
:10122000DF6E010E8FCFDBFF0BD08750DF6E010E1C
:1012300090CFDBFF05D08850DF6E010E91CFDBFF32
:101240006EDA0CDA9FDADFCFE6FFD1DA010EDB507F
:10125000DF5C0CE0E6DB4C0E65DA410E63DA540E1F
:1012600061DADFDB010EDBCFE6FFC1DA67DA020EFF
:10127000E15C02E2E16AE552E16E57D200DB05E192
:10128000DAC6E6FFDBC6E6FF39DB4FD252DA9FDA79
:10129000510E48DA90EC12F0EDDACAEC12F0E55299
:1012A000E552E66EA4DA4ADA40D23AEF0BF0E7DA1A
:1012B0000BE1E8DA300E36DA310E34DA2E0E32DA9D
:1012C000330E30DA320E79DB30D233DADEDA9EECEE
:1012D00049F0E5522AD22DDA040EE126030E73DB23
:1012E0003EE1000EDEC6DFFF010EDFC6DBFF020EB1
:1012F000DB6A030EDB6A97DA100E0B6E270E0C6E9C
:101300000D6A0E6AEECF06F0EECF07F0EECF08F0D2
:10131000EFCF09F038EC4BF005C0EDFF04C0EDFF56
:1013200003C0EDFF02C0EFFF7EDAEE52080EEE269C
:10133000000EEE22EE2277DA0C0EE76ED890030E46
:10134000EB32020EEB32010EEB32EF32E706F6E142
:10135000000EDFCFE6FF010EDBCFE6FFF2DA040E70
:10136000E15C02E2E16AE552E16EDFD177DB540A2B
:1013700011E0150A0AE07A0A11E142EC48F032DB8A
:1013800047EC48F0E552E55209D083DA07E1050160
:10139000E29D04D07EDA02E10501E28DC6D1B2DA27
:1013A00014CFDEFF15CFDDFFD6EC28F0000912E1E7
:1013B000030E09DB0AE0050E84DA0CE0CEDA0AE15E
:1013C00038EC0FF0000901E18EDAA0DA98EC48F071
:1013D000E552E552020EE15C02E2E16AE552E16E9D
:1013E000A4D14DDA05E100C6E6FF01C6E6FFA9DAA1
:1013F0009CD145DA05E1CFC6E6FFD0C6E6FFA1DA0B
:1014000094D13DDA08E13EDA30EC39F045DA3DDAE4
:1014100044EC35F053DA89D175DA040E52DA09E07A
:10142000070ED1DA06E1F4DACBEC11F0E552D2DAAC
:101430000BDB020EE15C02E2E16AE552E16E75D17E
:1014400059DA3B0803E136C7E6FF06D03DDA09E189
:1014500030DA07E0DFCFE6FF18DAE4EC3CF0E552E3
:10146000E552E55262D1D9CFE6FF5FD108DA06E155
:1014700009DA2050E66EBBD9A3DA07D025DA06E1F7
:10148000200EE66E000E58DAE552E5524ED13ADAF9
:10149000040E17DA09E0070E96DA06E1B9DAE1EC94
:1014A00011F0E55297DAD0DA020EE15C02E2E16A6D
:1014B000E552E16E3AD1E3D905E13EC7E6FF3FC709
:1014C000E6FFF3D932D1DBD904E1DCD9D6EC28F040
:1014D00047DA2BD12ED97BD9D8D96EEC3AF0E55228
:1014E00024D1CDD905E1A5DA200B01E0010E38DACF
:1014F0001CD11FD9040EE126E4D926E0070EFCD842
:10150000200822E1040EE66E080EF9D832D91CE05C
:101510000C0E59DA19E1E7D9080E09DAE552020E84
:10152000F3CFDBFF030EF4CFDBFFACD90EDA8FD99C
:10153000ACD953EC35F026D98AD9E8D995EC38F0F6
:1015400038D994EC49F0BAD9040EE15C02E2E16AC0
:10155000E552E16EEAD093D905E1BBC6E6FFBCC611
:10156000E6FFA3D9E2D08BD905E1BFC6E6FFC0C62E
:10157000E6FF9BD9DAD083D902E17CD996D9D5D0C0
:101580007ED905E1C5C6E6FFC6C6E6FF8ED9CDD039
:1015900076D905E1B9C6E6FFBAC6E6FF86D9C5D059
:1015A0006ED905E1BDC6E6FFBEC6E6FF7ED9BDD059
:1015B00066D905E1C3C6E6FFC4C6E6FF76D9B5D055
:1015C000D9CFE6FFB2D0B5D807014CA714D0050E8D
:1015D00078D911E0C2D90FE1030EA9D9E552F3CFB2
:1015E00000F6F4CF01F6020EE66E000EE66E060E71
:1015F000E66E000EC0D999D042D905E143D929C67B
:10160000E6FF1EDA15D045D913E12BDAE66E5CEC65
:1016100044F0E55200090CE0030E59D9EFCF29F64A
:10162000010EE66E290EE66E060EE66E290EA3D9B1
:101630007CD025D908E126D90001605102E1300EA5
:1016400001D0310EBAD971D074D8AAEC2DF05E0E4B
:1016500069D8010E51D866D8020E85D16AD812D940
:10166000030E81D166D857D9040E7DD1CAEC39F06A
:1016700094EF27F0AAEC2DF003D8F8DFFF0012005A
:10168000D0EC37F00009FCE1D8EC37F00009FCE1C0
:1016900012004FD8D6EC28F000091BE1D950FD0FFD
:1016A000E96EFF0EDA20EA6EEE50ED1001E1D6D8B9
:1016B00038EC0FF0000905E00F011451151101E09D
:1016C000CDD8FD0EDBCFE6FFE0D8DAEC28F0E5520E
:1016D000E5522BD07BD917EC35F0F0D826D076D94F
:1016E00044EC35F0EBD821D071D953EC35F0E6D885
:1016F0001CD06CD9A9D919D0EAD8EF501200E76EE6
:10170000FC0EDBCF14F0FD0EDBCF15F0E7501426F6
:10171000000E152214C0E6FF15C0E6FF120040D9E6
:1017200045EF0CF05FD9B6EF0CF0E552E7CFD9FFEB
:101730001200D9CFE6FFE1CFD9FF120041D9E5521F
:101740001200E76EFC0EDBCF16F0FD0EDBCF17F0BC
:10175000E7501626000E172216C0E6FF17C0E6FF58
:101760000BEC36F0E552E5524CEF0CF06DDFEEEF8E
:101770000CF0A2EC35F0DAEF0CF0146E050EE15E21
:10178000145012002BD911EF0DF02CD9CCEC34F001
:10179000E552E55212000BEC36F0E552E552F3CF7C
:1017A000DEFFF4CFDDFF1200D6EC1FF0E552DAEFDA
:1017B0000CF014D9EAEF0CF0FA0EDBCFE6FFFB0ECB
:1017C000DBCFE6FF45EF0CF0A1D845EF0CF05DD87C
:1017D00069EC38F0E5521200D9CFE6FFDACFE6FF28
:1017E000120053D898EC34F0E552E55212004DD86F
:1017F000A9EC34F0E552E552120069D8EFCF14F0AD
:10180000310E145C12002EDFE9D8DFCFE6FF1200A4
:10181000E66EE66A12EF3AF0E66EDFCFE6FF56ECD0
:101820001BF0E5521200D9CFE9FFDACFEAFF120030
:10183000E552DE52F3CFDEFFF4CFDDFFDD521200C2
:10184000010EDBCFE6FF020EDBCFE6FF1200020E39
:10185000DBCFE6FF030EDBCFE6FF1200FD0E14CF59
:10186000DBFFFE0E15CFDBFF1200D2EC35F0E552A8
:10187000E5521200C1C6E6FFC2C6E6FF1200DDD87F
:10188000E3EF0CF04CDFB6EF0BF0FE0EDBCFE6FF24
:101890001200040EE3EF0CF0F3CF14F0F4CF15F0C8
:1018A000F3CFE6FFF4CFE6FF120039DF1DDFBDEF17
:1018B0000BF092DF030E23DFD4EF0BF08FD89EEFF7
:1018C0000BF0E66E030EB2D0050EE3EF0CF0E76E00
:1018D000FC0EDBCFE9FFFD0EDBCFEAFFE750E92688
:1018E000000EEA221200030E0ADFCBEF0BF0B6D88F
:1018F000310A12001EDFE65231EF0DF010DFEADE92
:10190000BDEF0BF016DF020EE1261200DECFE6FF80
:10191000DDCFE6FF120003DFA1DEEEEF0CF054DFB7
:1019200062EC35F02FDF53DF440E92EF0BF0E7DE71
:101930000BEC36F0E5521200E66E030EE0DE35EFFA
:101940000CF0EDDED6DEBDEF0BF03EDF53EC35F0F4
:10195000C2EF0BF0060EE3EF0CF0080EE3EF0CF015
:1019600014DF9EEF0BF0C8DEDDDEDFD623EC38F0AF
:10197000E552E55212004CDFBDEF0BF0040EE66EAF
:10198000050E54D0B9DE48DFE552DF2A1200030EFF
:10199000E66E4CD0DFCFE6FF24DFDFCFE6FF12009C
:1019A000FC0EDBCFE6FFFD0EDBCFE6FF1200B7DE5D
:1019B00003EF0CF013D800091200B4DE9EEF0BF019
:1019C00064DF6CEF38F098DE3B081200B2DE5ADFBD
:1019D000DCEF0BF0E55260DF45EF0CF0E552E5522D
:1019E000E5521200E66E45EF0CF08CDF7CDF1BDF6A
:1019F000EE50ED10120096DE36C7E6FFF2DE86EFFF
:101A00000CF01BEC0FF0D5DE53EC35F05EEF0CF074
:101A10006ADF38DF9ADF86EF0CF08BDEE65259EF93
:101A20000CF033DF75EC38F0E552120068DEB9EFE8
:101A30000BF028DF07014C5112007BDE030E120071
:101A400024DF94DF9EEF0BF062EC35F05EEF0CF0DC
:101A5000C1DF53EC35F0C2DFE0EF0CF0EEDF7CEFDE
:081A60000BF0030E7CEF0BF00C
:081A680069EC13F00601A2EC89
:101A700013F002E2010E01D0000EE66E0601E05105
:101A80009CEC13F0E552E750EF6EE02B070EE017E9
:101A9000A2EC13F01DE2DF6A010EDB6ADB500808DE
:101AA0000AE0010EDB509CEC13F0EF5001E0DF2A5E
:101AB000010EDB2AF3D7DF5002080AE287AA06D01C
:101AC0004A0EE66E1CEC41F0E55202D007014B8154
:101AD000020EE15C02E2E16AE55232EF13F08AECB9
:101AE00013F010E20601DE2B000EDF2320AA4CD0FB
:101AF0006DEC13F050C6E6FF51C6E6FFB2EC13F0F2
:101B0000850E21D00601D8510601545D0601D95138
:101B1000060155591BE207014E510601685D070198
:101B20004F510601695912E20601DE2B000EDF2338
:101B300020AA2AD0B7EC13F0DEC6E6FFDFC6E6FF28
:101B4000F7EC13F0870E4DEC13F01CD00601DE51BC
:101B5000DF111AE0DE07000EDF5B20AA15D0DEC61B
:101B600014F00001156A070E1416145015100CE13C
:101B70006DEC13F0890EE66E3E0EE66E1CEC2DF059
:101B8000146E060EE15E14500601DA510601465D40
:101B90000601DB510601475907E30601000ED88014
:101BA000DE55100EDF553FE220AA26D0F7EC13F0E9
:101BB0008B0EE66E3E0E55EC13F068C6E6FF69C666
:101BC000E6FFB7EC13F05DEC13F08C0E14EC14F0A0
:101BD000BCEC13F075EC13F08E0EE66E3E0E55EC79
:101BE00013F06DEC13F046C6E6FF47C6E6FFB2EC15
:101BF00013F0950E14EC14F087BA0DD08AEC13F0A4
:101C000004E2B2EC13F0520E03D0B7EC13F0530E13
:101C10007AEC13F004D0560EE66E1CEC41F0E5525F
:101C20000601DE6BDF6BD8510601405D0601D9511C
:101C3000060141591AE220AA0BD05DEC13F040C610
:101C4000E6FF41C6E6FF80EC13F09F0E14EC14F0A3
:101C500087BA06D080EC13F0500E7AEC13F004D063
:101C6000460EE66E1CEC41F0E55206010251010BF6
:101C700005E14E0E07011B5D01E1F6DE1200D4EC1A
:101C800013F0E652DF6A080EDF5C06E0DF509CECE2
:101C900013F0EF6ADF2AF7D7E552DEEF13F027ECF7
:101CA00014F03CC7DFFF010E3DC7DBFF020EDB6A0D
:101CB000030EDB6ACBC614F0CCC615F046EC13F06D
:101CC000CBC60BF0CCC60CF085EC13F039EC13F05E
:101CD000640E0B6E0C6A0D6A0E6A20EC13F0F0ECC9
:101CE00013F0EE5C1550EE581650EE581750EE58A3
:101CF00009E3F0EC13F0EE5E1550EE5A1650EE5A72
:101D00001750EE5A000EDFCFE6FF010EDBCFE6FFE5
:101D1000C1EC13F02CEC13F0F3CFD1F6F4CFD2F6E4
:101D2000040EE15C02E2E16AE55232EF13F027ECC7
:101D300014F0D950FD0FE96EFF0EDA20EA6EEE5076
:101D4000ED1003E1F36AF46A27D0FDEC13F0000E06
:101D500014C0DFFF010E15C0DBFF020EDB6A030EAD
:101D6000DB6AEBEC13F0F30E0B6E0C6A0D6A0E6A75
:101D700039EC13F0080EE76ED890030EEB32020E2A
:101D8000EB32010EEB32EF32E706F6E1DFCF14F073
:101D9000DBCF15F018EC14F0040EE15C02E2E16A0E
:101DA000E55232EF13F00601D46BD56BD66BD76BCF
:101DB000C76BC86BD86BD96BDA6BDB6BDC6BDD6B1D
:101DC000120069EC13F0DE6ADD6A0601BF510701FB
:101DD0003A5D0601C05107013B5924E23A51060120
:101DE000BF5D166EC05107013B55176E0A0E086E97
:101DF000096A85EC13F0F2EC3EF006C014F007C05F
:101E000015F0210E1426000E1522420E0D6E0E6ADC
:101E100014C008F015C009F01FEC4CF008C0DEFF3C
:101E200009C0DDFF4AEC13F0020EE15C02E2E16A58
:101E3000E55232EF13F0DBDBFB0EDBCF14F0FC0ED0
:101E4000DBCF15F046EC13F014C00BF015C00CF00E
:101E500085EC13F020EC13F04AEC13F0040EE15C77
:101E600002E2E16AE55232EF13F09E9C4FEF0FF071
:101E700082BA000C0601D85106014E5D0601D95107
:101E800006014F5901E2010C0601DC5106014E5DCD
:101E90000601DD5106014F5901E2010C000C69EC0D
:101EA00013F0909A0F01239D9992C80EE66E45ECAF
:101EB0004CF0E55284EC4CF099820F01238D070E13
:101EC000E66E45EC4CF0E5520601B76BB86B30DBC3
:101ED000C5C6C7F6C6C6C8F6C5C6DEFFC6C6DDFFA0
:101EE000DDDAF3CFBBF6F4CFBCF6D9EC13F0060184
:101EF0001450F35C1550F45804E2BBC6DEFFBCC6B8
:101F0000DDFF20DBD9EC13F006011450C35D155042
:101F1000C45904E2C3C6DEFFC4C6DDFFC3DAF3CF93
:101F2000BDF6F4CFBEF6D9EC13F006011450F35C05
:101F30001550F45804E2BDC6DEFFBEC6DDFFF0DA80
:101F4000D9EC13F006011450C15D1550C25904E2DA
:101F5000C1C6DEFFC2C6DDFFC8DAD9EC13F0060148
:101F60001450B95D1550BA5904E2B9C6DEFFBAC6BD
:101F7000DDFF07014C9B46EC47F0000902E007013A
:101F80004C8BDECFB7F6DDCFB8F60F01239D9992CB
:101F9000020EE15C02E2E16AE55264D327EC14F040
:101FA000DF6A82BA03D007014D87DF8007014D51F8
:101FB00001E1E4D1918A4DB3908284EC4CF00701A9
:101FC0004DA51BD00601D451D51109E01DEC14F02C
:101FD000AEDEE552E552F3CFD4F6F4CFD5F60601E6
:101FE000D651D71109E022EC14F0A1DEE552E552FA
:101FF000F3CFD6F6F4CFD7F6FAD99ADA07014DA384
:1020000003D099820F01238D8BDA9CDA07014DBB37
:102010007EDA919A07014DA32BD0010EDB680F0EDB
:10202000F36E020EF3CFDBFF140EF36E030EF3CF4D
:10203000DBFF84EC4CF059DA010EDBCF14F0020E1A
:10204000DBCF15F006011450B95D1550BA5909E2FD
:10205000010EB9C6DBFF020EBAC6DBFF030EDB06BC
:10206000E8E1BEEC1BF00F01239D999273EC47F061
:1020700007014DBB43DA82AADF82030EDF5C02E078
:10208000DF500EE10601C151D45DC251D55901E2C4
:102090007DD9DF5005E1060102A1F1DD07014B9179
:1020A00007014DA902D015EC45F007014DA118D04C
:1020B000F5D906DBBBC6E6FFBCC6E6FFCDDAF3CF3B
:1020C000BBF6F4CFBCF6EED9FBDABDC6E6FFBEC662
:1020D000E6FFC2DAF3CFBDF6F4CFBEF63CEC1FF05C
:1020E00007014DAD17D0E2D9EBDA3EC7E6FF3FC797
:1020F000E6FFB2DAF3CF3EF7F4CF3FF7F350060135
:10210000305DF450315906E23EC7E6FF3FC7E6FFB7
:10211000540E2AD107014DAB31D1E1DC0601C75184
:10212000C8110DE1C5C6C7F6C6C6C8F6010E0F0B2D
:1021300010E0D890C833C733E806FBE10AD0C5C623
:10214000E6FFC6C6E6FF18DB87DAF3CFC7F6F4CFA3
:10215000C8F60601C751C81103E1DC6BDD6B08D07E
:102160000BDB2FD9E552E552F3CFDCF6F4CFDDF6E9
:1021700090A864D0215032E00601880E3C5D130E19
:102180003D592CE23CC614F03DC615F0070ECBDAE3
:10219000020E0F0B02E0FADAFEE10601DC51145CDC
:1021A000DD51155805E220AA42D02EDB440E3CD06A
:1021B0003AC614F03BC615F00B0EB5DA030E0F0B42
:1021C00002E0E4DAFEE10601DC51145CDD51155851
:1021D00035E220AA15D01EDB4E0E0FD087AA15D0EF
:1021E0000601DC5106013A5D0601DD5106013B594D
:1021F0000CE220AA05D00EDB580EE66E750E55DAFD
:10220000490EE66E1CEC41F0B0D087BA17D006013B
:10221000DC5106013C5D0601DD5106013D590EE22F
:1022200020AA05D0F1DA620EE66E750E3EDA5DDAAE
:10223000490E60DAE552BBEC44F0A0D0040E086E03
:10224000096AC9C60DF0CAC60EF0F2EC3EF006C02F
:102250003CF707C03DF70601CF51D01105E13CC75F
:10226000CFF63DC7D0F60AD03CC7E6FF3DC7E6FF34
:1022700092DAF2D9F3CFCFF6F4CFD0F60601CF51F0
:102280000601385D0601D0510601395903E283DAAF
:10229000480E6AD0020E0F01035D0CE106013651B3
:1022A0000601CF5D060137510601D05903E273DA0A
:1022B0004C0E5AD0DF500DE1BFC6E6FFC0C6E6FFA8
:1022C0003AC7E6FF3BC7E6FFC7D9F3CF3AF7F4CFEB
:1022D0003BF777DDF3CFCBF6F4CFCCF6F3CFE6FFC9
:1022E000F4CFE6FFCDC6E6FFCEC6E6FFB5D9F3CF05
:1022F000CDF6F4CFCEF6F3500601345DF4503559E7
:1023000006E2CDC6E6FFCEC6E6FF430E2DD0020E96
:102310000F01035D2FE1C3DC0601D1510601485DC9
:102320000601D2510601495922E20601D32BD351AD
:10233000190824E21A0ED36F20AA14D022DAE0D9A9
:102340003CC7E6FF3DC7E6FFCBC6E6FFCCC6E6FFCF
:10235000B50EE66E040EE66E5DEC2DF0146E0A0E00
:10236000E15E14500EDA440EC5D9E55207D00601DD
:10237000D36B04D00601D36BD16BD26B07014D6BCD
:10238000040EE15C02E2E16AE5526CD1E3D82FD899
:10239000EAD86FEF0DF02BD9E8C514F0E9C515F0B8
:1023A00075D9E8C50BF0E9C50CF03ADA03E0F3683B
:1023B000F46801D06FD9040EE15C02E2E16AE552F3
:1023C00051D115D9EAC514F0EBC515F05FD9EAC5AE
:1023D0000BF0EBC50CF024DA03E0F368F46801D0ED
:1023E00059D9040EE15C02E2E16AE5523BD10601F3
:1023F0000A0ED45D000ED55903E2D86BD96B06D016
:102400001CDACED9F3CFD8F6F4CFD9F606010A0EEE
:10241000D65D000ED75903E2DA6BDB6B120012DADD
:10242000BFD9F3CFDAF6F4CFDBF61200BDD9C26A1A
:10243000FE0EDB501F0BF36EF346F346830EC21401
:10244000F310C26EC16AFD0EDB50030BF36EF34650
:10245000F346F346F346CF0EC114F310C16EBA0E25
:10246000C06EC280C282C2B2FED7C290FF0ED880B8
:10247000C3540F0EC45403E2F36AF46A0ED006018B
:10248000C350B75DC450B85904E2B751C35EB851E8
:10249000C45AC3CFF3FFC4CFF4FF90D1E66A030E52
:1024A00034EF13F0E66A060E34EF13F0030EE66E17
:1024B000010E34EF13F078D9FB0EDBCF16F0FC0ED3
:1024C000DBCF17F0FD0EDB501624146EFE0EDB5032
:1024D0001720156E010E1426000E1522010E0F0B8B
:1024E00002E054D9FEE1A4D969D1030EE66E160EBE
:1024F000BBD8F3CFB9F6F4CFBAF61200030EE66EEE
:10250000020EB2D8F3CFBFF6F4CFC0F61200030E1E
:10251000E66E010EA9D8F3CFC9F6F4CFCAF61200C1
:10252000E66A090EA1D8F3CFC1F6F4CFC2F61200C5
:10253000E66AE66A7BDFE552E552F3CFC5F6F4CFF3
:10254000C6F61200E66A040E8FD8F3CFC3F6F4CFB6
:10255000C4F61200C1C6D4F6C2C6D5F6C3C6D6F6B6
:10256000C4C6D7F6120084DC000913E0A6D895ECA7
:1025700038F0E552E552E552E552F3CF4EF7F4CF8D
:102580004FF7E5EC47F0000904E04EC750F74FC79E
:1025900051F712009ED8FD0EDBCFE6FFFE0EDBCF1B
:1025A000E6FFFED8F3CFDEFFF4CFDDFF320EDE26EE
:1025B000000EDD2210D9640E0D6E0E6AEECF08F00B
:1025C000EDCF09F01FEC4CF008C0EEFF09C0EDFFA5
:1025D000010EDB5002E0FF0E01D0DF50146E020E40
:1025E000E15C02E2E16AE552E16E1450E7D02FD9D6
:1025F000FD0EDBCF18F0FE0EDBCF19F01A6A1B6A56
:10260000FCD8166A176A14C006F015C007F016C089
:1026100008F017C009F018C00BF019C00CF01AC070
:102620000DF01BC00EF038EC4BF002C0DEFF03C013
:10263000DEFF04C0DEFF05C0DDFFDD52DD5212000B
:10264000C1D8CBEC4BF009C0EDFF08C0EDFF07C0CF
:10265000EDFF06C0EFFF12002EDFE552E552E55216
:10266000E5521200E16EAAD0E66EE0DEE552E552D8
:102670001200A8D838EC4BF005C0EDFF04C0EDFF08
:1026800003C0EDFF02C0EFFFEBEF13F0166A176A0D
:10269000EBEF13F08ED818EF14F0E66E3E0EE66EF8
:1026A0005DEC2DF0146E0A0E1200E66E1CEC2DF09F
:1026B000146E060EE15E14501200C4D81DEF14F023
:1026C000F3CF14F0F4CF15F0F3CFE6FFF4CFE6FF2D
:1026D00012006AD8020EE1261200E66A100EE66EBB
:1026E000DEC6E6FFDFC6E6FF1200DCC6E6FFDDC69B
:1026F000E6FF1200E66E4DEC32F0E552E5521200B4
:10270000D8C6E6FFD9C6E6FF120016C00DF017C006
:102710000EF012000601DA510601505D0601DB5190
:102720000601515912001502F3CF15F01402F3CF30
:1027300014F0F45015261200EA6AE10FE96E060E55
:10274000EA221200D8510601445D0601D951060162
:1027500045591200D950020FE96EDACFEAFFEE5068
:10276000ED101200DAC6E6FFDBC6E6FF12004EC728
:10277000E6FF4FC7E6FF1200C7C6E6FFC8C6E6FF82
:102780001200D1C6E6FFD2C6E6FF1200D89015327D
:102790001432E8061200CFC6E6FFD0C6E6FF1200EC
:1027A000FADDE552E5521200D9CFE6FFE1CFD9FFBD
:1027B0001200DECF14F0DDCF15F01200E552E7CFA6
:1027C000D9FF1200EECF06F0EECF07F0EECF08F003
:1027D000EFCF09F01200D9CFE9FFDACFEAFF1200FC
:1027E000D8C614F0D9C615F051DF1450120054C6E3
:1027F000E6FF55C6E6FF80EF13F0FD0EDBCF14F0C9
:10280000FE0EDBCF15F012003CC6E6FF3DC6E6FF2C
:1028100075EF13F03AC6E6FF3BC6E6FF75EF13F01F
:1028200074DF0EDFAAEF13F038DFE15E1450120000
:1028300014C0F3FF15C0F4FF1200D4C6E6FFD5C6DE
:10284000E6FF1200D6C6E6FFD7C6E6FF1200ACDFF1
:06285000040EE126120057
:0A285600BFEC18F0E6EC18F008E201
:1028600054EC19F0800EE926060E9BEC19F002D00C
:10287000F36AF46AC4EF18F0BFEC18F0030EE12617
:10288000D8EC19F0DF6EDFCFE6FFE5DFE552DE5270
:10289000D1EC18F0DD5220AE08D0CDEC18F0E66A8D
:1028A000BAEC18F0E70E23EC19F0010E3CEC19F02D
:1028B0000BEC19F0030EE15C02E2E16AE552E16E15
:1028C000C4EF18F0BFEC18F0050EE126DE68DD68F5
:1028D00003EC19F05F0ED880EE54EA0EED5407E2D7
:1028E0005F0EF36EFD0EF3CFDBFFEA0E11D0FD0E8F
:1028F000DBCF14F0FE0EDBCF15F0DC0E145C050E02
:1029000015580AE2DC0EF36EFD0EF3CFDBFF050E69
:10291000F36EFE0EF3CFDBFFD8EC19F0E76E020E7C
:10292000E7CFDBFF20A209D0BAEC18F0020EDBCF14
:10293000E6FFE66A220EA2EC19F00B0EF36E020E11
:10294000DBCFF4FFF350F45C3CE2020E42EC19F0F2
:10295000E66ED950030FE96EDACFEAFFE552E75091
:10296000EE6EED6A020EDB5006E103EC19F0DC0EB0
:10297000EE5E050E0ED0020EDB04E66E49D9E5527E
:10298000F3CF14F0F4CF15F003EC19F0F350EE5E32
:102990001550ED5A5BEC19F0030EDBCF0DF0040E71
:1029A000DBCF0EF01FEC4CF008C0DEFF09C0DDFFEE
:1029B00020A207D0DFEC18F0D6EC18F0250EA2EC20
:1029C00019F066EC19F00BEC19F0050EE15C02E26F
:1029D000E16AE552E16ED8D3D2DBE6EC18F009E209
:1029E000FE0EDB50EA6A960FE96E060EEA22EF5001
:1029F00001D0140EC9D3C3DBD8EC19F0E66EECDFBE
:102A0000E552C2D3BCDBFE0EDB500F0803E0AFEC97
:102A100019F00FD0FE0EDB6ADB500B0809E0AFECBB
:102A200019F0000902E1000E04D0FE0EDB2AF4D7F3
:102A3000010EAAD3A4DBFD0EDB50020A0FE0030A4D
:102A40000BE0010A0FE1010E2CEC19F0000902E184
:102A5000000E09D0020E03D0010E01D0020E2CECA4
:102A600019F001D0000E90D38ADB090EE126AEDB0F
:102A70004DE2FD0EDBCFE6FF7BEC47F0E5520009AF
:102A800045E082AA43D06BEC19F0E5DEE552020E78
:102A9000F3CFDBFF030EF4CFDBFFDE6ADD6A020E4D
:102AA000DB50DF1804E1030EDB50DE52DD1835E0A9
:102AB000FD0EDBCFE6FF7ADB6BEC19F0A8DB070E2F
:102AC000F3CFDBFF080EF4CFDBFF030EE66ED95029
:102AD000040FE66E000EDA20DBDBBCEC19F016E129
:102AE000040EDB50FF0808E1050EDB50FF0804E18F
:102AF000060EDB50FF080CE0030EE66E5B0EE66E82
:102B0000070EC6DBE0EC27F069DB02E0000E06D022
:102B1000DF2A010EC4E3DB2AC2D7010E146E090EB0
:102B2000E15C02E2E16AE552E16E14502DD327DB4D
:102B3000070EDADB010EE76E9FDBE7501426000E6E
:102B40001522030E14C0DBFF040E15C0DBFFDFCF20
:102B5000E6FF81DEE552050EF3CFDBFF060EF4CF74
:102B6000DBFF010E89DB0001800E151412E1F1DBA1
:102B700014DB83DA5ADB000942E075DB05E0010E65
:102B8000DBCF14F0020E1DD0010EDB06020E01E2B7
:102B9000DB062ADBE8AE02D0173404D01650145CF2
:102BA0001750155817E2D5DB0ADBDFCFE6FF65DAF1
:102BB0003CDB000924E057DB08E0030EDBCF14F018
:102BC000040EDBCF15F027DB1CD0030EDB2A040E2E
:102BD00001E3DB2AD950010FE96EDACFEAFFFF0EDD
:102BE000EE18BFE1FF0EED18BCE1FEDAE8AE02D050
:102BF000173404D01650145C17501558B2E3F3681C
:102C0000F468070EE15C02E2E16AE552E16EBCD2D3
:102C1000B6DA4ADBA10EE926060E8DDBB5D2B9DBAA
:102C2000DE6ADD6AD3DA2AE2FE0EDB5005E1DC0E55
:102C3000DE6E050EDD6E06D0FE0EDB04E66EE8DF0E
:102C4000E552AFDAFE0E1EDB166E176AFC0EDBCF06
:102C500008F0FD0EDBCF09F016C00DF017C00EF026
:102C6000C5EC3EF006C014F007C015F0D9CFE9FF5F
:102C7000DACFEAFF0650EE261550ED2220A208D04A
:102C800095DA2DDBFE0EDBCFE6FFE66AE90EDBDA36
:102C90001DDBC1DA020EE15C02E2E16AE552E16E9F
:102CA00073D26DDAFB0EDB04186E196A18BE196850
:102CB000020E086E096AFC0EDBCF0DF0FD0EDBCFB5
:102CC0000EF0C5EC3EF006501824166E0750192081
:102CD000176E030E1702F3CF17F01602F3CF16F09C
:102CE000F4501726E60E1A6E980E1B6E000E1C6E20
:102CF000FE0EDBCF1DF01E6A1F6AD8901D361E36F1
:102D00001F361A501D24F36E1B501E20F46E1C50EB
:102D10001F20F86EF4CFF7FFF3CFF6FF0900F55050
:102D20001624146E0900F550172014C0F3FFF46E3A
:102D30002BD225DA030ED8DA3EDA2FDA68DA030E60
:102D4000E15C02E2E16AE552E16E1ED218DA040E9D
:102D5000E12614CFE6FF15CFE6FF4DDEE552E55242
:102D6000DE6EDD6AFD0EDBCF16F0FE0EDBCF17F058
:102D70000F011650145D175015590BE3FD0EDB5073
:102D8000145D0001146EFE0EDB500F011559000199
:102D900006D091DA1451085C146E15510958156E5D
:102DA000020E14C0DBFF030E15C0DBFF020EDBCFEB
:102DB00014F0030EDBCF15F0DECF18F0DDCF19F0E5
:102DC000DE501824166EDD501920176E1450165C54
:102DD0001550175802E3000E18D020A215D0E6D9DE
:102DE000020EDBCFE6FF030EDBCFE6FF14CFE6FFDC
:102DF00015CFE6FFBFD9EB0EE66EE66A5DEC2DF06F
:102E0000146E0A0EE15E1450010E146E040EE15CA5
:102E100002E2E16AE552E16E1450B6D1BADA20A2BC
:102E200014D0FC0EDBCF14F0156A14BE156814C064
:102E3000E6FF15C0E6FF9ED9510EE66EE66A1CEC71
:102E40002DF0166E060EE15E1650B5D97BEC47F0FC
:102E5000E552000904E0D7D9EE50ED1002E1000E72
:102E60002BD0E20EE66E050EE66E97DA60DE146E8B
:102E7000050EE15E145095D929DA0001800E151473
:102E800004E00501E26BE36BE46BFD0EDBCFE0F5E4
:102E9000FE0EDBCFE1F520A20ED0E4C5E6FFE3C5D0
:102EA000E6FFE2C5E6FFDFCFE6FF520EE66EE66A1A
:102EB0009DEC2DF0BAD9010E146E020EE15C02E217
:102EC000E16AE552E16E14505FD159D9050EE12651
:102ED0002BDAC7EC4AF02BDA02DAA2D9DF6E58D926
:102EE000DFCFE6FFF8D903EC20F0E552E5520B0EF8
:102EF000DF5C2DE2F4D954DA010EE66EF0D919DF69
:102F000016DA030EF3CFDBFF040EF4CFDBFF07016D
:102F10004CA704D0F7D953D9DED98CD939D9420E70
:102F200022D9490E20D94E0E1ED91FDAD4D944EC2D
:102F300035F0FDD932D9CFD97FD8F9D9E552010E74
:102F4000E66E3DD97BD9020EE66E39D977D9050EEA
:102F5000E15C02E2E16AE552E16E16D110D9E1507E
:102F6000B1D9800B01E0010EE66EB5D906EC48F050
:102F700007DAD950A7D9400B03E0010EE66E01D065
:102F8000E66AA9D960EC48F0FBD915D9A4D955EC6B
:102F900043F0F6D9EFD8CFEC42F0E552E552F4D049
:102FA000EED8030EE126FB0EDB50020807E1D950F4
:102FB000FC0FEAD9030EEE26000EED22030EE66E9C
:102FC000D9CFE6FFDACFE6FF8AD9D6D92EE183D969
:102FD0006FEC38F0E55264D97ED9A0EC47F0E552A9
:102FE000E55207014CA705D09FD942D8E552E552DA
:102FF000E552CED8FF0EDF5C0EE1450EB4D84D0E83
:10300000B2D8500EB0D8540EAED8590EE66E63D971
:1030100023EC38F008D0DECFE6FFC8D8DD525BD90C
:103020009DDFE552E552E552E552030EE15C02E216
:10303000E16AE552E16EA8D0ACD932D950D9EFDDC2
:1030400076D9AFD8A5D8460E8ED8520E8CD8B3D923
:103050002D0E89D8FD0E16D9FF0FDE26000EDD22BB
:10306000AAD9020EE15C02E2E16AE552E16E8CD07F
:1030700086D848D959D9DED887D03CD9F90EDBCFCC
:10308000E6FFFA0EDBCFE6FF91D876D902E1010E1A
:1030900001D0000E146E020EE15C02E2E16AE5521C
:1030A000E16E145071D06BD88BEC3FF007C0E2F5A5
:1030B00008C0E3F509C0E4F507C0E6FF08C0E6FF75
:1030C00009C0E6FF6AD927D8B0D85ED076EC47F0C1
:1030D000E66EE66A87EC47F0E552E552E66AEBEC0D
:1030E00047F0E55242EC48F0E66EE66A47EC48F0FD
:1030F000E552E55231EC43F0E66EE66A46EC43F009
:10310000E552E552ABEC42F0E66EE66AC0EC42F006
:10311000E552E55212003DD940D90BDE08D941D81D
:10312000030EE66ED950F90FF6D802E1010E01D078
:10313000000E146E020EE15C02E2E16AE552E16EFD
:10314000145022D0D7D8D950F80FE5D802E1010E9B
:1031500001D0000E146E020EE15C02E2E16AE5525B
:10316000E16E145011D0E66EB6D823EC38F0E5527B
:10317000E5521200FD0EDBCFE6FF6BEF19F0D9CF61
:10318000E6FFE1CFD9FF1200E552E7CFD9FF1200E9
:10319000A2D875EC38F0E5521200E7D8DFCFE6FF91
:1031A0001200F3CFDEFFF4CFDDFF1200DECFE6FF2B
:1031B000DDCFE6FF1200FC0EDBCFE6FF1200030EB0
:1031C000DBCFE6FF040EDBCFE6FF12000B0EF36E43
:1031D000FE0EDBCFF4FFF350F45C1200146E050E0C
:1031E000E15E145000091200030EDBCF14F0040E50
:1031F000DBCF15F0050EDBCF16F0060EDBCF17F098
:10320000155017181200D950FD0FC4EF19F049DD01
:103210008ED8E552120014C0F3FF15C0F4FF12005F
:1032200066EC1DF0E552E5521200146E060EE15EEA
:103230001450120062EC35F097EF19F04CD8B0DE64
:1032400076D8E5521200E66EE66A3CEC2DF0146E7C
:10325000080EE15E14501200E66E3DD834EC15F015
:10326000E552E5521200FA0EDBCFE9FFFB0EDBCF91
:10327000EAFFEF50FF081200DBCF14F0020EDBCFA5
:1032800015F01200DBCFE6FFECEC14F0E552120073
:10329000E66E070EDBCFE6FF080EDBCFE6FF12007F
:1032A000FB0EDBCFE6FF1200FE0EEA6ADB34FE0BFC
:1032B000EA36E96E1200FD0EDBCF08F0FE0EDBCF22
:1032C00009F01200FB0F60D8EF501200DECF14F0AF
:1032D000DDCF15F01200FE0EDBCFE6FF12006BDF34
:1032E000FD0EDBCFE6FF1200E12662D8DF6E42DF83
:1032F000D0EF19F04ED8D4DF50D889DF52DF030E5B
:10330000E66E1200410E2FDF440E2DDF440E2BDF40
:10331000520EB3EF18F0E66EFF0EDA20E66E46DFCF
:10332000E0EC27F0EEEF18F033DFCDEF19F0E552C7
:10333000E552E5521200EA22EECF14F0EFCF15F07D
:103340000BEF19F0E66E010EE66E1CEC2DF015EF9A
:1033500019F0FA0EDBCFE6FFA3DFDBEF18F00ADF90
:103360001AEC15F0E552E5521200010EDBCFE6FF34
:10337000020EDBCFE6FF1200B3EC27F0EEEF18F001
:10338000E552E552C8EF18F0E96EFF0EDA20EA6E5A
:103390001200F5DE020EE12612000DDFBAEF18F082
:1033A00062EC14F0E552E552DE52FBDEDD52120013
:0E33B000E1DE10EF19F0FADE8EDF1AEF19F0F1
:0233BE001DDB15
:1033C00036C7DFFF0701366B0B0E365D04E00AD807
:1033D0000701362BF9D7DFCFE6FF92EC1FF0E5525D
:1033E000E552C7D26EDB080EE12608D9000967E076
:1033F0004BDB29DB200EE66EE66AE6680ADBEFECC3
:103400004BF0146E050EE15E14500501200EDC6FCA
:10341000030EDD6F420EDE6F36C7DFF5E06BE16B4A
:10342000E26BE29FE29DE36BE46B010EE56F030E3E
:10343000EE6F2ADBEECFE6F5EECFE7F5EECFE8F55F
:10344000EECFE9F5EECFEAF5EECFEBF5EECFECF50A
:10345000EFCFEDF5400EE66F010EE76F580EE85D19
:10346000020EE95906E3B00ED880E855040EE9557E
:103470000BE2120E146E980E156E000E83DAF5CF65
:10348000E8F50A00F5CFE9F5DC0EEA5D050EEB592B
:1034900006E3980ED880EA55080EEB550BE2280E8D
:1034A000146E980E156E000E6DDAF5CFEAF50A006F
:1034B000F5CFEBF5FF0EEC5D01E1EC6BE2D9080E08
:1034C000E15C02E2E16AE552E16E53D2F7DA03E130
:1034D000EEC5DFFF04D0010E28DA120E2EDA030E3D
:1034E000DF14E55246D2EADA03E1ECC5DFFF04D08F
:1034F000010E1BDA100E21DAC7DAEF50010B02E0E1
:10350000010E01D0000EE55234D2AEDA05E1E0C57D
:10351000DEFFE1C5DDFF04D0020E07DA040E0DDA8E
:10352000B3DAEE50ED100AE1FE0EDBCFE6FF53EC0E
:103530001FF0E552F3CFDEFFF4CFDDFF20A60DD064
:10354000DECFE6FFDDCFE6FFFE0EDBCFE6FFE66A6D
:10355000E70EE66E030EE66E61DA46DA020EE15C15
:1035600002E2E16AE552E16E04D2A8DA03E1050164
:10357000ED5105D0010ED9D9110EDFD9DF50E5523A
:10358000F8D172DA05E1E8C5F3FFE9C5F4FF05D02B
:10359000020ECBD90C0ED1D927DA020EE15C02E281
:1035A000E16AE552E16EE5D15FDA05E1EAC5F3FFD4
:1035B000EBC5F4FF05D0020EB8D90E0EBED914DA51
:1035C000020EE15C02E2E16AE552E16ED2D107014E
:1035D000366B0B0E365D05E016D853D90701362B36
:1035E000F8D712000501E26BE36BE46B120008DA16
:1035F00002E3000E02D0DED95ADABBD136C7E6FFAD
:1036000008DAEAEF1CF0FADF000901E1000C0DD93D
:1036100000090EE120500BE0000EE66EE66A07019D
:103620003651E66EE66A700EE66EE66AF7D9DADEC5
:10363000010CE3D9C8D9EF50800B01E0010EE66E12
:1036400017EC48F0E552DF6EBED9EF50400B0BE0AF
:10365000010EE66E6DEC48F0E552DF5C02E1000E13
:1036600007D0010E05D0E66A6DEC48F0E552DF1296
:10367000AAD9EE52EF50E66E5FEC43F0E552DF124E
:10368000A2D9020EE926000EEA22EF50E66ED9EC2E
:1036900042F0E552DF12DF50E5526BD1E20EE66EEA
:1036A000050EE66EC6DFE552E552120057D942E23A
:1036B000FD0EDB94DB96DB98DB9ADB9CDB9EDB501C
:1036C00039E00601D85106014E5D0601D9510601C7
:1036D0004F5930E352D902E1F5D801D0DAD9FD0EC5
:1036E000DB50E76E120EE7CFDBFF090EDB50020A5C
:1036F00007E0030A0DE199D9010B0AE1020E04D09B
:1037000094D9020B05E1010EF36E090EF3CFDBFF36
:10371000C3D933D90FE1FD0EDBCFEEF576EC47F0E0
:10372000146E090EDB50145C05E0090EDBCFFCF0D3
:103730000001FA81200EE15C02E2E16AE552E16EED
:1037400018D10CD914E219D909E1BCD80501EC91C2
:10375000FD0EDB5001E0EC8111D801D09AD9100E9A
:10376000DB90FD0EDB5002E0100EDB8095D9200EC1
:10377000E15C02E2E16AE552E16EFBD00501ECA1F9
:1037800002D09092120090821200E8D80FE2F5D891
:1037900005E198D8FD0EDBCFEDF501D07AD9FD0E0D
:1037A000DB50E76E110EE7CFDBFF76D9200EE15C30
:1037B00002E2E16AE552E16EDCD0D0D813E2DDD856
:1037C00008E180D8FC0EDBCFE8F5FD0EDBCFE9F594
:1037D00001D05FD931D90C0E08C0DBFF0D0E09C036
:1037E000DBFF5AD9200EE15C02E2E16AE552E16EAC
:1037F000C0D0B4D813E2C1D808E164D8FC0EDBCF46
:10380000EAF5FD0EDBCFEBF501D043D915D90E0E4D
:1038100008C0DBFF0F0E09C0DBFF3ED9200EE15CC4
:1038200002E2E16AE552E16EA4D00501DC51146EBA
:10383000156A200E145C000E155801E2000C030EF0
:10384000DD5D01E0000C420EDE5D01E0000C0701D1
:1038500036510501DF5D01E0000CE5C5E6FF7BECBC
:1038600047F0E552000901E1000C200EE66ED1D8C8
:103870006EEC4AF0E552E552E552000901E0000C19
:10388000010C36C7E6FFC5D8EFEF1CF0B9D819E236
:103890001F0E05D96EEC4AF0E552E552E552FF0DD8
:1038A000F350E66E90D81F0EE926000EEA22E5528C
:1038B000E750EF6E7FD812EC3AF0166E050EE15E1F
:1038C000165057D0E1D8DCC5EEFFDDC5EEFFDEC5F2
:1038D000EEFFDFC5EEFFE0C5EEFFE1C5EEFFE2C59E
:1038E000EEFFE3C5EEFFE4C5EEFFE5C5EEFFABD8A6
:1038F000EEC5EEFFEFC5EEFFF0C5EEFFF1C5EEFF42
:10390000F2C5EEFFF3C5EEFFF4C5EEFFF5C5EEFF21
:10391000F6C5EEFFF7C5EEFFF8C5EEFFF9C5EEFF01
:10392000FAC5EEFFFBC5EEFF1200E66ED9CFE6FF4B
:10393000DACFE6FFFE0E39EF1DF01426000E152239
:1039400014C0E6FF15C0E6FF57EF1DF0FE0EDBCFFB
:10395000E6FFD9CFE6FFDACFE6FF1200B2D8200E9D
:10396000E1260B0EF36EFE0EDBCFF4FFF350F45C9A
:103970001200E552E7CFD9FF1200FE0EDB5007011F
:10398000365D1200166E36C717F0186A196AD8909D
:1039900017361836193614501724F36E15501820A0
:1039A000F46E16501920F86EF4CFF7FFF3CFF6FF40
:1039B00009001200200E73D8FC0E5BD814C0E6FF7D
:1039C00015C0E6FF1200FD0EDBCFE9FFFE0EDBCFD8
:1039D000EAFF12000CDEE552E552E552120056DF16
:1039E000E552E552E5521200DECF14F0DDCF15F0BE
:1039F00014C0F3FF15C0F4FF120063D8E6521200A2
:103A000060D80B0EF36EFC0EDBCFF4FFF350F45CCA
:103A10001200DC0EE66E050EE66E12001CEC2DF0B8
:103A2000146E060EE15E14501200D950120FE96EAA
:103A3000DACFEAFFEF501200FC0EDBCF08F0FD0EEC
:103A4000DBCF09F01200E6C5EEFFE7C5EEFFE8C5E3
:103A5000EEFFE9C5EEFFEAC5EEFFEBC5EEFFECC5F4
:103A6000EEFFEDC5EEFF12002CD8020EE126BDEFF1
:103A70001CF0DB50200DF3CF14F0F4CF15F0000E46
:103A80001426010E15221200D9CFE9FFDACFEAFF82
:103A900012005CDFEAEF1CF059DFEFEF1CF0E66E7E
:103AA000FD0EDBCFE6FFFE0EDBCFE6FF1200F1ECF2
:103AB00039F0166E050EE15E165012009EDFBDEF66
:0C3AC0001CF0D9CFE6FFE1CFD9FF1200C7
:043ACC00D1DAE65213
:103AD0000F0EDF6EA3DADC0E145C050E155858E3EA
:103AE0009DDA680E145C420E15582AE297DA700EC1
:103AF000145C170E155812E291DAB80E145C0B0E16
:103B0000155802E2DF6A44D089DA940E145C110E73
:103B1000155802E2010E3BD0020E39D07FDA280E92
:103B2000145C230E155802E2030E31D077DAC80E6A
:103B3000145C320E155802E2040E29D0050E27D06F
:103B40006DDA900E145C650E155812E267DA380EC5
:103B5000145C4A0E155802E2060E19D05FDAD80E30
:103B6000145C590E155802E2070E11D0080E0FD042
:103B700055DA700E145C940E155802E2090E07D047
:103B80004DDA600E145CEA0E155802E20A0EDF6E82
:103B900078DA55D9E552E552DF50E5526ED206018A
:103BA0002951440A08E01D0A04E0100A0EE1E6EF7C
:103BB0001DF08EEF1EF00001605101E00F0C8DDA58
:103BC00002E2E6EF1DF08EEF1EF00F0C51DA090E47
:103BD000E126DF6ACD0EF36E070EF3CFDBFF0C0E8E
:103BE000F36E080EF3CFDBFF78DA06E2070EBDC6F0
:103BF000DBFF080EBEC6DBFF010EBBC6DBFF020EFD
:103C0000BCC6DBFF030EDB6A040EDB6AD950010F72
:103C1000E96EDACFEAFFCD0E0B6E0C0E0C6E0D6A5C
:103C20000E6A3BDA38EC4BF005C0EDFF04C0EDFF47
:103C300003C0EDFF02C0EFFF070EDBCF14F0080E4C
:103C4000DBCF15F0166A176AD950010FE96EDACF8B
:103C5000EAFF14C00BF015C00CF016C00DF017C031
:103C60000EF01BDACBEC4BF009C0EDFF08C0EDFF06
:103C700007C0EDFF06C0EFFF010EDBCF08F0020E1C
:103C8000DBCF09F0050E08C0DBFF060E09C0DBFF25
:103C9000050EDBCF14F0060EDBCF15F0400E196ECB
:103CA000970E1A6E000E1B6EDFCF1CF01D6A1E6A87
:103CB0002CDA1CC007F01DC008F01EC009F010EC83
:103CC0003FF004C01CF005C01DF006C01EF01950E6
:103CD0000424F36E1A500520F46E1B500620D6D92A
:103CE000F5CF16F00900F5CF17F00800F5CF18F062
:103CF0001450165C1550175802E2DF2AC9D7400E3F
:103D0000146E970E156E000E90D9146E090EE15CBC
:103D100002E2E16AE552E16E1450AFD1A9D9E65250
:103D2000DF6A5B0E176E970E186E000E196EDFCFEE
:103D30001AF01B6A1C6AE9D91AC007F01BC008F008
:103D40001CC009F010EC3FF004C01AF005C01BF0D5
:103D500006C01CF017500424F36E18500520F46EB2
:103D60001950062093D9F5CF14F00900F5CF15F0BE
:103D70000800F5CF16F00601BB51145CBC51155874
:103D800002E2DF2ACED75B0E146E970E156E000E80
:103D90004CD9E55272D1B3D902E08FD902E3000EBB
:103DA00015D094EC46F041EC1CF020A80CD0FE0E8F
:103DB000DBCFE6FFE66A07013651E66EE66A140ECF
:103DC000E66E1E0E82D997D9ADD8E55256D150D99C
:103DD000E65212CFE6FF13CFE6FF78DEE552E5525A
:103DE000DF6EDF98DF9ADF9CDF9E07016851DF5CA2
:103DF0001FE107013651DF5C05E00F0EDF5C02E0DA
:103E0000010E396F0F01035113E107013951040A03
:103E10000CE0050A03E0010A0BE009D0DFCFE6FF62
:103E2000BADFE5520701392B03D0396B01D0392BAA
:103E3000DFCF68F70F01126B136BE5521ED118D953
:103E400053D908E6900E145C650E1558000E1658EE
:103E5000000E17580BE348D908E6600E145C6D0E8F
:103E60001558000E1658000E175803E307014B971C
:103E700002D007014B8701D1FBD8E65290DEDF6EFE
:103E8000DF500701345D04E0DFCF34F7356B09D034
:103E90003551146E156AFF0E141801E1155001E03A
:103EA000352BE552EAD0E4D87F0E166E970E176ECA
:103EB000000E186EFE0EDBCF19F01A6A1B6AD8903E
:103EC00019361A361B3616501924F36E17501A205D
:103ED000F46E18501B20DAD8F5CF14F00800F5CF97
:103EE00015F014C0F3FF15C0F4FFC7D0070134511B
:103EF000375D01E1000C040E355D01E2000C0B0E94
:103F0000345D01E3000C20A80AD03451E66EE66A65
:103F10003751E66EE66A600EE66E1F0ED6D834C7DD
:103F200037F7010CECD802E0C8D802E3000E3DD010
:103F300006014A510601DC5D06014B510601DD59BF
:103F400003E20F01146B156BFE0EDBCF36F703ECAB
:103F50001BF007014CB304D0CED8DAEC40F0E552A8
:103F6000BEEC1BF020A81CD036C7E6FFE66A3DD8A1
:103F7000E552E552E0C5E6FFE1C5E6FFE5C514F010
:103F8000156A14BE156814C0E6FF15C0E6FF620E80
:103F9000E66EE66A1CEC2DF0166E060EE15E16501B
:103FA0000601FC6BDEEC32F0010E67D061D8FB0E2F
:103FB000DBCFE6FFFC0EDBCFE6FF63D8B7EC35F0D6
:103FC000E552E552E552E55200090DE0FB0EDBCF6C
:103FD000E9FFFC0EDBCFEAFFEFCF14F00B0E145C11
:103FE00002E2010E01D0000E48D042D884D869EC1C
:103FF00038F0E55246D807D8E552E5527CD86CEC4B
:1040000038F0E5523AD034D8420E50D84E0E4ED841
:1040100038D898EC34F0E552E5522FD0FD0EDBCFC6
:1040200014F0FE0EDBCF15F01200166EDFCF17F086
:10403000186A196A6AD817C007F018C008F019C0C2
:1040400009F010EC3FF014500424F36E15500520D5
:10405000F46E16500620F86EF4CFF7FFF3CFF6FF9C
:10406000020EF626000EF722F8220800F550120084
:10407000D9CFE6FFE1CFD9FF1200E552E7CFD9FF54
:104080001200FD0EDBCFE6FF7BEF20F0F86EF4CFE1
:10409000F7FFF3CFF6FF09001200EECF06F0EECFE8
:1040A00007F0EECF08F0EFCF09F01200E66E23D84C
:1040B00023EC38F0E552E55212000B0EF36EFE0EC3
:1040C000DBCFF4FFF350F45C1200E66E1CEC2DF035
:1040D000146E060EE15E145012000601F40ED88034
:1040E000BD55090EBE55120099DF166A176AD890A1
:1040F0001750000A1200FE0EDBCFE6FF1200B8DFF9
:10410000FE0EDB500701365D1200030E0C6E0D6AC9
:044110000E6A120021
:0C411400D9CFE6FFE1CFD9FF51DA3B081C
:1041200004E158DA6CEC38F036D24ADA5E0801E085
:1041300033D2010E3DDA580A01E113D20F0A01E130
:1041400003D2010A01E1D5D1020A01E192D1070AA5
:1041500001E160D1010A01E14DD1030A01E146D13B
:10416000010A01E11DD11F0A01E112D1020A01E198
:1041700001D1010A01E1E8D0060A01E1DDD0030A1C
:1041800001E1D6D00E0A01E1CBD0010A01E1A5D0B0
:10419000030A71E0010A55E0070A4BE0010A23E037
:1041A000030A01E0F9D10FDA540A19E0060A13E014
:1041B0001C0A0DE00B0A07E0010A01E0EDD1F0D97D
:1041C0003BEC04F0E6D1ECD946EC04F0E2D1E8D9BE
:1041D000ADEC04F0DED1E4D9D6EC04F0DAD1E0D9CC
:1041E00005EC05F0D6D1EFD9590A1FE0010A19E014
:1041F0000A0A13E01C0A0DE00D0A07E0020A01E0BA
:10420000CBD1CED91FEC05F0C4D1CAD94EEC05F004
:10421000C0D1C6D985EC05F0BCD1C2D9C0EC05F03F
:10422000B8D1BED91FEC06F0B4D1BAD95CEC06F017
:10423000B0D1C9D9520A01E0AFD1B2D977EC06F0BA
:10424000A8D1C1D9500A13E01D0A0DE0040A07E005
:104250000F0A01E0A1D1A4D991EC06F09AD1A0D91E
:10426000ABEC06F096D19CD9CEEC06F092D198D961
:10427000E4EC06F08ED1A7D9570A2BE0030A25E01B
:10428000060A1FE0020A19E01D0A13E0040A0DE005
:104290000F0A07E0050A01E07FD182D907EC07F099
:1042A00078D17ED927EC07F074D17AD943EC07F0A6
:1042B00070D176D95BEC07F06CD172D97AEC07F04B
:1042C00068D16ED9BFEC2FF064D16AD990EC07F0B9
:1042D00060D166D905EC30F05CD175D9540A19E08B
:1042E0001A0A13E0020A0DE0090A07E07E0A01E05B
:1042F00053D170D9ABEC07F04ED152D9B7EC07F0DF
:1043000048D14ED9C1EC07F044D14AD9D4EC07F0DA
:1043100040D15CD901E040D15DD9F4EC07F03BD14C
:1043200052D94F0A01E038D13BD9FFEC07F031D127
:1043300037D909EC08F02DD146D9410A01E02CD13A
:104340002FD95FEC25F025D13ED9520A0FE01B0A88
:1043500009E00D0A01E020D139D901E01DD125EC99
:1043600008F01AD11DD92CEC08F013D119D947EC5B
:1043700008F00FD128D9540A07E0100A01E00CD147
:104380000FD960EC08F005D10BD96FEC08F001D122
:104390001AD9500A01E000D103D982EC08F0F9D013
:1043A00012D9560A1FE0060A19E0190A13E00F0A8B
:1043B0000DE0020A07E0070A01E0EED0F1D8ACEC0C
:1043C00008F0E7D0EDD8B4EC08F0E3D0E9D8BCECC5
:1043D00008F0DFD0E5D8CCEC08F0DBD0E1D8D4ECA5
:1043E00008F0D7D0DDD83EEC09F0D3D0F3D846ECB6
:1043F00009F0D1D0E8D8560A09E0050A01E0CCD08E
:10440000E5D801E0C9D055EC09F0C6D0C9D857ECC1
:1044100009F0BFD0D8D8570A28E0010A22E0180ACC
:104420001CE0030A16E0040A10E00A0A0AE0010A86
:1044300001E0B2D0CBD801E0AFD0CCD865EC09F028
:10444000AAD0AED86BEC09F0A4D0AAD8B6EC09F08B
:10445000A0D0A6D8CFEC09F09CD0A2D8F1EC09F0FE
:1044600098D09ED8F9EC09F094D09AD801EC0AF0D3
:1044700090D0A9D8570A39E0020A33E0060A2BE0A7
:10448000030A25E01D0A1FE0040A19E00C0A13E0E4
:10449000010A0DE0060A07E0030A01E07DD080D89A
:1044A0000CEC0AF076D07CD820EC0AF072D078D8E8
:1044B00033EC0AF06ED074D836EC0AF06AD070D8BB
:1044C00047EC0AF066D06CD85BEC0AF062D068D892
:1044D00063EC0AF05ED07AD85FE17CD86AEC0AF02F
:1044E0005AD05ED871EC0AF054D05AD879EC0AF060
:1044F00050D069D8560A24E0040A1EE01F0A18E0CA
:10450000040A12E00F0A0CE0020A06E0060A44E17F
:1045100047D8ABEC0AF03DD043D8B3EC0AF039D021
:104520003FD8BBEC0AF035D03BD8C0EC0AF031D014
:1045300037D8C8EC0AF02DD033D8D0EC0AF029D007
:104540002FD8D8EC0AF025D03ED8530A06E0180A36
:1045500023E126D8E0EC0AF01CD022D8E3EC0AF0E4
:1045600018D031D8590A12E0010A0CE0080A06E016
:10457000190A12E115D8FCEC0AF00BD011D819EC8D
:104580000BF007D00DD89AEC25F003D009D80AEC2F
:1045900026F0E552E552E552E552E7CFD9FF120089
:1045A000FC0EDBCFE6FFFD0EDBCFE6FFEAEF22F0ED
:1045B000E76E14D8E750E926000EEA22EF50120009
:1045C0000DD8EF501200020ED8EF22F0030EF0DFEC
:1045D0003B081200FE0EDBCFE6FF1200FC0EDBCF25
:0A45E000E9FFFD0EDBCFEAFF120039
:0645EA00070155A323D0D8
:1045F0005593205002E0830E08DA0501E551020AC6
:1046000005E0030A07E10001020E02D00001010EDD
:10461000FC6FFA8120500FE0FCC014F0156A14BE44
:10462000156805DAE5C516F0176A16BE17682FDAA1
:10463000830EF2D931DA12000001FAA156D0FA91B4
:1046400011DA0601D8510601425D0601D951060171
:1046500043590CE220AA49D042C6E6FF43C6E6FF12
:10466000D8C6E6FFD9C6E6FF8C0E1DD00001FC05BA
:104670000BE10501EE51010B07E1205036E0F9D9BD
:1046800014AE0FD015680DD0020E0001FC5D0FE1D5
:104690000501EE51020B0BE1205027E0EAD914BED0
:1046A0001568C5D98D0EB8D9060EE15E120000015D
:1046B000FC510501E55D19E020500FE0FCC014F04D
:1046C000156A14BE1568B3D9E5C516F0176A16BE8B
:1046D0001768DDD98E0EA0D9DFD9FCC0E5F541EC15
:1046E0001CF0E9D902E00001FA8B1200D9CFE6FFF5
:1046F000E1CFD9FFE65282BA0BD00F011451151148
:1047000009E014CFFEF015CFFFF00001FA8702D0C8
:104710009EEC28F00001FAA721D0FE51FF111EE007
:10472000C0D966EC1DF0E552E552DF6EDFCFE6FF43
:10473000CBEC1EF0E552000911E020A807D0B1D95A
:10474000DFCFE6FFE66AA20E67D9B0D907EC41F0E9
:104750000601FC6BB0D902E00001FA8BE552E5528C
:10476000E7CFD9FF1200070155A10CD0559138ECC5
:104770000FF0000907E176D9205002E0790E45D903
:1047800094EC41F0120097D929E006014A51060144
:10479000DC5D06014B510601DD5920E30F01145188
:1047A00015111CE00501E0510F01141904E1050188
:1047B000E1510F01151912E048D9A6EC16F0E552A7
:1047C000E55200090BE020A608D03FD914CFE6FF40
:1047D00015CFE6FFA90E20D969D92ED912000701FD
:1047E00055A507D055950001FA89205002E0960E94
:1047F0000CD91200B8DFF9DE1FDFF1DF77DF070128
:104800004CBB04D00001FA6BFB6B12000001FA51A3
:10481000100B03E150D901E0B6DF0001FAA910D076
:1048200020A602D0B40EF1D8A6EC41F0420805E172
:104830004D0EE66EDBEC41F0E552DEEC32F00BD0D3
:1048400018EC29F0000909E020A602D0BE0EDDD840
:10485000F3D80001FA8307014C9D010E216E00017F
:10486000FAAB23D0FA9B20A60BD0000EE66EE66AC8
:1048700018D9120EE66E020EE66E1CEC2DF016D95B
:104880000001FAA70AD0FE51FF1104E0FEC0E0F5D6
:10489000FFC0E1F5FA97FE6BFF6BE5C5E6FFD5D8E3
:1048A0000EEC17F0E552E552E5520001FA51100BFB
:1048B00003E130D8000906E077EC45F020A629D0C6
:1048C000260E22D018EC29F0000908E020A602D01C
:1048D000350EC0D80001FA89FA8312000001FAA946
:1048E00004D020A616D03A0E0FD014D8000904E048
:1048F00020A60FD0440E08D0090E216E0001FAA5A3
:1049000005D020A606D0570E2AEF25F037EC45F04B
:10491000216A1200E5C5E6FF7BEC47F0E55200098D
:1049200005E176EC47F00501E56F010C76EC47F008
:104930000501E55D17E020A614D0E5C514F0156A61
:1049400014BE156874D876EC47F0166E176A16BE5A
:1049500017689DD8220EE66E030EE66E1CEC2DF055
:104960009BD8010CA6EC41F0420804E00501E2519D
:10497000800B07E1580EE66E070E82D801E0000CAE
:10498000010CE20EE66E050E7BD801E0000C010C76
:10499000D9CFE6FFE1CFD9FFE150FD0FE96EFF0E61
:1049A000DA20EA6EEE50ED102BE085D829E038D8F9
:1049B000CBEC3AF0E552E55233D866EC1DF0E55207
:1049C000E552E66ECBEC1EF0E552E5C5E6FF28D8D1
:1049D0000EEC17F0E552E552E552000911E020A671
:1049E0000DD0E5C514F0156A14BE156820D82DD871
:1049F000CF0E12D8166E060EE15E1650010E01D0D3
:104A0000000EE552E7CFD9FF1200E66EE66A06EC2B
:104A10002DF0E552E5521200E66EE66A1CEF2DF02D
:104A2000FD0EDBCFE6FFFE0EDBCFE6FF120014C06B
:104A3000E6FF15C0E6FF120014CFE6FF15CFE6FF34
:104A4000DAEC28F0E552E5521200E0C5E6FFE1C5D8
:104A5000E6FF1200E66E020EE66E06EC2DF0E55261
:104A6000E5521200DEEC32F007EC41F00601FC6B7F
:104A70001200EE51E66EE66AFCC014F0156A1200F0
:104A8000E66E59EC3FF0E552E5520009120016C0FF
:104A9000E6FF17C0E6FF1200186E060EE15E185022
:104AA0001200FEC0E6FFFFC0E6FF1200146E060E05
:0E4AB000E15E14501200A9EC41F00009120062
:024ABE006AD9B3
:104AC000030E08D93B080FE187D924EC0BF0E5521F
:104AD000E552E552060102B102D0350E52D9300E30
:104AE00050D98CD926D0030EE66E040EE66E990ED0
:104AF000E66E000E26D903E0060102910BD0070EE8
:104B0000E66EFC0EE66E980EE66E000E1AD911E007
:104B100006010281020EE66E020EE66E060EE66EDB
:104B2000020EE66EE66A12EC3AF0146E050EE15ED5
:104B3000145035D15BD95A0A58E0030A54E0010AEF
:104B400050E00F0A4CE0010A48E0030A44E0010A81
:104B500040E0070A3CE0020A38E0010A34E01E0A9D
:104B600030E0030A2CE0010A28E0070A24E0010AE9
:104B700020E0020A1CE00F0A18E0010A14E0030A10
:104B800010E0010A0CE0070A08E0010A04E0030A49
:104B90003AE1300E2BD0320E29D0340E27D0360E0B
:104BA00025D0380E23D03A0E21D03C0E1FD03E0E19
:104BB0001DD0400E1BD0460E19D0480E17D0420E05
:104BC00015D04A0E13D04C0E11D0500E0FD04E0EF1
:104BD0000DD0600E0BD0620E09D0640E07D0660EA9
:104BE00005D06A0E03D0680E01D0440EDE6EDD6A79
:104BF000DAD809E0DFD802E17AD805D007014CA75E
:104C000002D08AD8B6D8040EE15C02E2E16AE5522D
:104C1000E16EC5D0EBD8430A0AE0010A04E0030ABA
:104C200027E1540E01D0020EDE6EDD6A16D06C0E46
:104C3000DE6EDD6A040E4ED83B080FE06DD8F3CF70
:104C400014F0F4CF15F0F3CFE6FFF4CFE6FF16EC47
:104C50004BF0E552E55200090BE0A5D809E0AAD8CF
:104C600002E145D805D007014CA702D055D881D81C
:104C7000040EE15C02E2E16AE552E16E90D08AD86E
:104C8000F90EDBCFF3FFDB06F350000921E0FD0E48
:104C9000DBCFE9FFDB2AFE0EDBCFEAFF01E3DB2AF5
:104CA000EFCF14F0D950FA0FE96EFF0EDA20EA6E5A
:104CB000EFCFF6FFEE2AEFCFF7FF000EEE22EFCF99
:104CC000F8FFEE220800F550145CDAE0000E01D087
:104CD000010E65D0E76EFC0EDBCFE9FFFD0EDBCFEA
:104CE000EAFFE750E926000EEA22EF50120074D8DE
:104CF0002EEC0BF0E552E552E55287D8EECFE6FFF9
:104D0000EFCFE6FFFE0EDBCFE6FF62EC35F0E552BB
:104D1000E552E552FEEF26F0040EE76EFC0EDBCF07
:104D200016F0FD0EDBCF17F0E7501626000E172207
:104D300016C0E6FF17C0E6FF0BEC36F0E552E55271
:104D40001200E66E030EE76EFC0EDBCF14F0FD0ED4
:104D5000DBCF15F0E7501426000E152214C0E6FF35
:104D600015C0E6FF8CDF166E060EE15E16500009D8
:104D70001200F4CF15F049D8F3CFEEFF15C0EDFFC8
:104D80001200E66EFE0EDBCFE6FF23EC38F0E552B4
:104D9000E5521200D9CFE6FFE1CFD9FF1200E5526C
:104DA000E7CFD9FF1200D9CFE9FFDACFEAFFEE5003
:104DB000ED101200DECF14F0DDCF15F0000E14263A
:104DC000060E1522020E14C0DBFF030E15C0DBFF1A
:104DD000040E80DF3B081200FC0EDBCFE6FFFD0E69
:104DE000DBCFE6FFFE0EDBCFE6FF1200D3DF040EC3
:104DF000E126DE6ADD6A030E6AEF26F0FE0EDBCFE7
:104E0000E6FF6CEC38F0E5521200020EDBCFE9FF52
:084E1000030EDBCFEAFF1200E4
:084E180045D9020EE126DF6A14
:104E20007FD9EE50ED102EE0DE52400EDD6E60D9DF
:104E3000400E145C000E155806E2FB0EDB50E76EC8
:104E4000010EE7CFDBFF010E12D91CE15FD908E1AB
:104E5000FD0EFE0EDBCF15F052D902E15CD903E066
:104E6000E4EC43F00FD0010EDBCFE6FF15D8E5529E
:104E7000DF6EE4EC43F0DF5005E1E4D8EE5E155060
:104E8000ED5ACED7DF50146E020EE15C02E2E16A09
:104E9000E552E16E14500BD105D9E652FE0EDBCF80
:104EA000F3FFDB06F350000905E0E668C5D8F6E03D
:104EB000DF5001D0000EE552FAD0F4D8FCD8000E35
:104EC000145C400E155811E213D9FD0EDBCF16F01D
:104ED000FE0EDBCF17F0000ED8801656400E175688
:104EE0001450165C1550175802E2000E01D0010E46
:104EF000DED0D8D8E6523F0EE76EFD0EDBCF14F0C1
:104F0000E7501416156A400ED8801456000E155638
:104F10001450DF6EFC0EDB50DF5C02E2DF5002D08B
:104F2000FC0EDB50E552C3D0BDD8E652DF6A84ECFC
:104F30004CF0DAD8A1B612D0C5D808E0C5AC0AD07A
:104F4000DCEC43F0A1B60AD0BDD8F8E1E4EC43F0C4
:104F5000FD0E07D0E4EC43F0A1A602D0FF0E01D075
:104F6000000EE552A4D09ED8E652DEDFDF6EDF50A1
:104F700024E18CD802E1F70E21D0C8D81AE19BD8E1
:104F8000BED817E1C8D815E1DCEC43F0A10EE66EFF
:104F900053D805E0E4EC43F0BCEC43F00ED0FA0E3D
:104FA0009AD8F9EC43F0E552E552E552DF6EC6ECD3
:104FB00043F0E4EC43F084EC4CF0DF50E55277D062
:104FC00071D8020EE126DF6A61D802E1F70E2BD01C
:104FD000FA0EDB5027E0FA0E4AD824E197D805E113
:104FE0006AD88DD802E197D803E0E4EC43F01AD0F8
:104FF000010E71D811EC44F0E552E552E552DF6E36
:10500000E4EC43F0DF500EE11DD8EE261550ED2202
:10501000FA0EDBCFE7FF010EDB50E75EFA0EE7CFBB
:10502000DBFFD6D7DF50146E020EE15C02E2E16ACC
:10503000E552E16E14503BD0E8EC43F0E552DF6EF0
:10504000DF501200010EDB50146E156AD950FD0FAF
:10505000E96EFF0EDA20EA6E1450EE261550ED22AE
:10506000010EDB50146E156A5BD814501200DBCFB2
:10507000E6FF5DD83EDFE552E552E552E76E010EF0
:10508000E7CFDBFF51DFDF6EDF501200FA0EDBCF20
:10509000E6FFE66A4CD811DFE552E552E552E552EB
:1050A00000091200D9CFE6FFE1CFD9FF1200E55287
:1050B000E7CFD9FF1200FD0EDBCF14F0FE0EDBCFE1
:1050C00015F01200A00EE66EE8EC43F0E552DF6E3C
:1050D000FF0EDF5C1200DBCFE6FFFB0EDBCFE6FF4F
:1050E000FC0EDBCFE6FF1200BCEC43F0E0EF43F038
:1050F000FB0EDBCF14F0FC0EDBCF15F0120015C059
:1051000014F0156A1450E66E1CEF28F0EDDFA00EC7
:10511000E66E1CEF28F0FD0EDBCFE6FF1CEF28F05B
:10512000D950FB0FE96EFF0EDA20EA6E1200FD0E79
:0C513000DBCFE6FFFE0EDBCFE6FF120037
:04513C0076EC1FF0FE
:1051400000091EE0070136510701375D19E037C736
:10515000E6FF85EC1AF0E552F3CFFEF0F4CFFFF056
:105160000001FA8720A80CD0FEC0E6FFFFC0E6FFD2
:1051700007013751E66EE66AA30EE66EE66A29D9A4
:1051800012000001FA51040B03E1070155510DE033
:105190000701556B20A608D0040EE66E290EE66EB8
:1051A00006EC2DF0E552E552010C000C215001E116
:1051B000000C010C36D9E150FD0FE96EFF0EDA202C
:1051C000EA6EEE50ED1015E020A60AD014CFE6FFEF
:1051D00015CFE6FF0DD93C0EE66E280EE66EF9D827
:1051E000FD0EDBCFFEF0FE0EDBCFFFF00001FA87F5
:1051F000FA8B1CD1E0C5FEF6E1C5FFF6E5C5FDF66C
:1052000020A615D0FDC614F0156A14BE156814C08A
:10521000E6FF15C0E6FFFEC6E6FFFFC6E6FFD20EBC
:10522000E66E280EE66E1CEC2DF0060EE15E120016
:1052300007014CAB000CA6EC41F0410801E0000C6A
:105240004E0E07011B5D01E0000C06014A510601EC
:10525000DC5D06014B510601DD5901E2000C0F0136
:105260001451151101E1000C07014E510601605D5A
:1052700007014F510601615901E3000C20A60CD033
:1052800060C6E6FF61C6E6FF4EC7E6FF4FC7E6FF12
:10529000C00EE66EE66A9DD876EC47F00601FD5D2D
:1052A00014E1FEC6E6FFFFC6E6FFA6EC16F0E552E7
:1052B000E55200090AE107014E510701605D07014F
:1052C0004F510701615901E3000CA0EC3AF0010CC9
:1052D000A8D8FE0EDBCFE6FF7BEC47F0E5520009D5
:1052E00007E076EC47F0146EFE0EDB50145C02E132
:1052F000000E39D020A61ED0FE0EDBCF14F0156AAA
:1053000014BE156814C0E6FF15C0E6FF76EC47F042
:10531000166E176A16BE176816C0E6FF17C0E6FFBE
:10532000D80EE66E270EE66E1CEC2DF0186E060EFB
:10533000E15E185077EC45F0000903E00F010351DE
:105340000AE15DD80AE220AA06D062D8E20EE66E33
:10535000270EE66E3ED8010E06D0FE0EDBCFE6FF2E
:10536000ACEC47F0E55262D05CD842D859EC3FF043
:10537000E552E552000902E0000E2AD077EC45F034
:10538000000907E020A602D0830E2AD80F0103519E
:1053900018E135D809E220AA14D03AD8850EE66E75
:1053A000270EE66E16D80DD023D819EC1BF0E55267
:1053B000E552000908E020AE04D0880E11D866EC52
:1053C00018F0010E05D0205002E0920E09D8000E10
:1053D0002DD01CEC2DF0146E060EE15E1450120060
:1053E000E66E270EE66E06EC2DF0E552E552120051
:1053F000FD0EDBCFE6FFFE0EDBCFE6FF120006015F
:10540000D8510601425D0601D951060143591200E7
:1054100042C6E6FF43C6E6FFD8C6E6FFD9C6E6FFAA
:105420001200D9CFE6FFE1CFD9FF1200E552E7CF56
:04543000D9FF12008E
:0C54340007014CA90AD03F0E8112C00EE7
:1054400083126C0E841287800F0E881202D031D81E
:1054500021D985D876EC47F0010802E18D88120049
:105460008D98120007011B51480A21E01C0A1DE01B
:10547000070A19E0010A17E0020A13E0110A13E013
:105480000D0A15E0050A0BE00C0A11E0010A05E01F
:10549000070A01E012008A8212008A8202D08A88FA
:1054A00012008A8612008A8A12008A8412008A8078
:1054B00012000701662B6651A20801E2666B8C9E02
:1054C000020E0F01035D01E18C8E919007014CA546
:1054D0000AD04E0E07011B5D04E17C0E0701665DDC
:1054E00004E2918002D087AA9180C00E8A1691961C
:1054F000919491924E0E07011B5D07E07C0E07010F
:10550000665D2CE2918232EF2AF007014BA106D0B2
:105510007C0E0701665D22E28A86120006012B518D
:10552000010B0BE007014B5108E18250200B05E114
:10553000100EE66E270EE66E04D0D8C6E6FFD9C67A
:10554000E6FF1FD8E552E552D6EC28F0000906E048
:105550008A9A7C0E0701665D01E28A8A1200A6EC37
:1055600041F0410A0BE0030A06E00F0A01E01200D5
:10557000FC0E8C1612008C928C8012008C908C8207
:105580001200D9CFE6FFE1CFD9FFBFD8680E145C77
:10559000290E155802E3918406D0B7D8800E145C0A
:1055A000250E155802E3918606D0AFD8980E145CEC
:1055B000210E155802E33F0E8A12A7D8B00E145CD4
:1055C0001D0E155802E33E0E37D09FD8C80E145C4E
:1055D000190E155802E33C0E2FD097D8E00E145C3C
:1055E000150E155802E3380E27D08FD8F80E145C2C
:1055F000110E155814E289D8A00E145C0F0E155820
:1056000004E3030E070166150AE17FD8AC0E145CB3
:105610000D0E155806E3010E0701661502E1300E66
:105620000BD073D8B80E145C0B0E155807E3030E9D
:105630000701661503E1300E8A1228D066D8D00E15
:10564000145C070E155814E260D8DC0E145C050ECD
:10565000155804E3030E070166150AE156D8E80E53
:10566000145C030E155806E3010E0701661502E1EE
:105670008A8A0CD04AD806014E51145C4F511558F5
:1056800005E3010E0701661501E18A8AE552E7CFBD
:10569000D9FF1200D9CFE6FFE1CFD9FF020EE126F4
:1056A000930E8D16909006014C510601D85D0601AF
:1056B0004D510601D9591FE330EC39F0F3CFDEFF2D
:1056C000F4CFDDFF29D81E0E2CD801E3908024D81A
:1056D000140E27D801E38D8C1FD80F0E22D801E3BA
:1056E0008D841AD80C0E1DD801E38D8A15D80A0EA8
:1056F00018D801E38D86020EE15C02E2E16AE55210
:10570000E16EE552E7CFD9FF1200FD0EDBCF14F0BA
:10571000FE0EDBCF15F01200DECF14F0DDCF15F05A
:0A5720001200145C000E1558120070
:06572A003AD9E652FAC66E
:105730002AF7FBC62BF7F9C6E6FFF9D8E5520701B1
:10574000296F50D9F9C6E6FFCBD8E552E5520701DB
:10575000266FDFCFE6FFF9C6E6FFAED8E552E55289
:105760000701276F20A60AD027C7E6FF26C7E6FF56
:1057700029C7E6FFF9C6E6FF330E2BD926C7F9F68F
:10578000F8C6E6FFD4D8E5520701286F2BD9F8C632
:10579000E6FFA6D8E552E5520701246FDFCFE6FF0A
:1057A000F8C6E6FF89D8E552E5520701256F20A625
:1057B0000AD025C7E6FF24C7E6FF28C7E6FFF8C6DC
:1057C000E6FF350E06D924C7F8F60601060EE96F86
:1057D000080E0701275D09E20601ECB306D0EC8351
:1057E0000601F76B0601090EE96FE552DED0D8D845
:1057F000020EE12620EC42F0070125510601F85D7A
:105800000EE2F8510701255DDF6E2851D880DF5484
:1058100002E228C7DFFFDF500601F8272FD007017B
:1058200027510601F95D17E2F9510701275DE76E7F
:10583000010EE7CFDBFFDBCF14F02951D8801454E1
:1058400003E2010E29C7DBFF010EDB500601F92739
:1058500024C7F8F613D0F7510DE10601EC51040B03
:1058600009E1EC850601010EF76F24C7F8F626C79B
:10587000F9F604D050EC42F00601EC81020EE15C36
:1058800002E2E16AE552E16E90D08AD8E652FE0E5D
:10589000DB50DF6E06010D0E8CD801E277D80601D1
:1058A0000F0E87D801E272D806011E0E82D801E2DF
:1058B0006DD8DF50E55279D073D8FD0EDB50146EF1
:1058C000156AFE0E7BD8E8AE02D0173404D016500D
:1058D000145C1750155802E28CD801D0FF0E65D029
:1058E0005FD8FE0EDBCF14F0FD0EDB50D8801454D1
:1058F00008E2FE0EDBCFE6FFFD0EDB50E552E75C73
:1059000001D0000E52D04CD8FE0EDB50146E156A3A
:10591000FD0E54D8E8AE02D0173404D01650145CF3
:105920001750155802E265D801D0FF0E3ED038D886
:1059300006010D0E3ED804E364D8E842070B0CD0F4
:105940000F0E37D803E35DD80F0B06D0140E31D8F5
:1059500008E357D8E8461F0BE76EFE0EE7CFDBFFE4
:105960000BD0050E146E0E6EFE0EDBCF09F065EC4B
:105970004CF0FE0E09C0DBFFDB5005E1010EF36EBB
:10598000FE0EF3CFDBFFFE0EDB500FD0FE0EDBCFA3
:10599000E6FFDFCFE6FFB7DFE552E552DF6E12002C
:1059A000D9CFE6FFE1CFD9FF1200E552E7CFD9FF0B
:1059B0001200D880FA55000EFB551200DB50166E0F
:1059C000176AFF0ED8801656000E17561550171876
:1059D0001200E66EE66A9DEC2DF0146E060EE15E96
:1059E00014501200E66E51DFE552DF6EDFCFE6FFA6
:1059F0001200FD0EDBCFE6FFFE0EDB50E552E72482
:0C5A00001200FE0EDBCFE7FFE7381200BB
:045A0C00F0D80FE1DE
:105A1000FE0EDB5015180BE1E70E07012E1902E10F
:105A2000030E2F1904E02E2B000E2F2304D092D842
:105A30000FD9E9D82DD9ECD0DAD81BE1FE0EDB5016
:105A4000151817E1EED815E1FC0EDB50171811E11F
:105A5000F0D80FE1FA0EDB5019180BE1E70E070141
:105A60002E1902E1030E2F1904E02E2B000E2F2316
:105A700002D091D8C8D8CCD0BAD81BE1FE0EDB50EA
:105A8000151817E1CED815E1FC0EDB50171811E1FF
:105A9000D0D80FE1FA0EDB5019180BE1E70E070121
:105AA0002E1902E1030E2F1904E02E2B000E2F23D6
:105AB00003D071D8B1D8A7D8ABD099D81BE1FE0ECE
:105AC000DB50151817E1ADD815E1FC0EDB501718A7
:105AD00011E1AFD80FE1FA0EDB5019180BE1E70E18
:105AE00007012E1902E1030E2F1904E02E2B000EE0
:105AF0002F2308D050D890D8F50EDBCFE6FFF60E56
:105B0000BED881D885D0ABD8FA0EDBCF32F7FB0EEA
:105B1000DBCF33F79DD878EC38F0FC0EDBCFE6FF17
:105B200090D8FB0EACD86FD873D0BFD8FE0EDB5028
:105B3000206E6ED049D867D86BD046D878EC38F054
:105B4000780EE66E7ED893D8F90EDBCFE6FFA7D8A5
:105B50005AD85ED006EC3BF007012E512F111AE007
:105B6000B1D8520E90D82CC7E6FF2DC7E6FFA3D8B8
:105B70000701010ED8802E55000E2F5505E22EC7C5
:105B8000E6FF2FC7E6FF97D83ED807012E6B2F6B95
:105B90002C6B2D6B1200DEDF7BD8FB0EDBCF30F7DA
:105BA000FC0EDBCF31F7F90EDBCF32F7FA0EDBCF8D
:105BB00033F74ED8FB0EDBCFE6FFFC0E60D8F90EB4
:105BC000DBCFE6FFFA0E59D04AD8FB0EDB50326F1E
:105BD000336B3ED878EC38F0780E55D8FC0EDBCF1E
:105BE000E6FF45D8FB0EDBCFE6FF4FEF2EF0D9CF17
:105BF000E6FFE1CFD9FF2CC714F02DC715F0FD0E3D
:105C0000DB5014181200E66A6CEC38F0E552120012
:105C1000E552E7CFD9FF1200F70EDBCFE6FFF80E13
:105C20002CD030C716F031C717F0FB0EDB5016181A
:105C3000120032C718F033C719F0F90EDB501818EC
:105C4000120038EC38F0E552FA0EDBCFE6FF120016
:105C500039D8FD0EDBCFE6FFFE0E3FEF2EF025D844
:105C600017D8FC0EDB500701306F316B120017D8CC
:105C700078EC38F0780E43EF2EF03FEF2EF0DBCFCC
:105C8000E6FF5BEF2EF0E66E38EC38F0E5521200DE
:105C9000FD0EDBCF2CF7FE0EDBCF2DF71200E66AF0
:105CA000A9EC34F0E552E5521200D9CFE6FFE1CF7E
:105CB000D9FFAAEF2DF0E66A3AEC35F0E552E5524D
:0E5CC000E5521200540EDFDF500E43EF2EF0BF
:025CCE000001D3
:105CD000FA51020B16E007014E510601605D070103
:105CE0004F51060161590DE320A609D060C6E6FFB9
:105CF00061C6E6FF35D9920EE66E130E21D9090E64
:105D000001D0060E216E120077EC45F0000904E088
:105D10000F01035101E0120007014CBD0AD0E66AF1
:105D200017EC48F0E552000904E020A68AD0C80E1E
:105D30001CD006014A510601DC5D06014B510601EB
:105D4000DD5916E220AA7DD0DC51DD110DE04AC6F6
:105D5000E6FF4BC6E6FFDCC6E6FFDDC6E6FFE60E65
:105D6000E66E0F0EA0EF2FF0E60EE66E0F0E09D0D6
:105D70000F011451151106E120A663D0040EE66E42
:105D8000100EF3D0E8D866EC1DF0E552E552E66E51
:105D9000CBEC1EF0E552000916E0DDD81FEC1FF039
:105DA000E552E55220A808D0000EE66EE66AD3D888
:105DB000360EE66E100EC4D8CED8DAEC28F0E552D6
:105DC000E552216A1200C7D8C3EC3AF0E552E55219
:105DD000E5EC47F0000928E007014C8D20A604D02F
:105DE000E66A9EEC49F0E552070150510601645DF8
:105DF000070151510601655917E320AA0CD064C66A
:105E0000E6FF65C6E6FF50C7E6FF51C7E6FF0E0E88
:105E1000E66E100E95D8F2EC1AF04EEC1BF0B8ECD2
:105E200048F0090E216E1200B5EC3EF094D8C8EC93
:105E300024F0E552E5520501E28F4EEC1BF0050E11
:105E4000216E12004E0E07011B5D05E020A653D007
:105E50007A0E7ED850D00601ECA141D014CFE0F5E7
:105E600015CFE1F5FAEC28F007014E5106016A253D
:105E70000701606F07014F5106016B210701616F38
:105E8000060160510701605D06016151070161591A
:105E900004E260C660F761C661F720A607D060C75C
:105EA000E6FF61C7E6FF5CD88E0E65D8070150514A
:105EB00007014E5D0701515107014F590DE320A61F
:105EC00007D04ED850C7E6FF51C7E6FF910E53D812
:105ED000F2EC1AF04EEC1BF0B8EC48F00CD0C1EC30
:105EE00028F000090BE020A602D0990E31D89BECD7
:105EF00042F04EEC1BF0090E216E1200010EE66E10
:105F000017EC48F0E552000905E020A618D09D0ED8
:105F1000A8EF2FF038EC0FF000090DE120AA0FD008
:105F20004EC6E6FF4FC6E6FFD8C6E6FFD9C6E6FF77
:105F3000B60EBBEF2FF02EEC3EF04EEC1BF0120035
:105F4000E66E1CEC2DF0146E060EE15E145012008D
:105F5000E66E170E0AD014CFE6FF15CFE6FF12004B
:105F60004EC7E6FF4FC7E6FF1200E66E06EC2DF0C7
:0E5F7000E552E5521200E66E170EA0EF2FF07C
:025F7E0015D933
:105F800029E027D927E02CD925E005019A5122E004
:105F90009A5140081FE3DB0EE66E050EE66E0A0E10
:105FA000A9D818E033D9DB2515E10C0EBCD83B0885
:105FB00011E1030EB8D8530A08E0030A0BE1C0D878
:105FC000F1EC39F0CCD808E105D0BAD8B3EC27F021
:105FD000C6D802E0000E14D0D0D8DF6A05019A516D
:105FE000DF5C0BE0DF50EA6A9B0FE96E050EEA22E8
:105FF000EF50E66E90D8DF2AF1D7A8D81424E1D864
:10600000E552E552E7CFD9FF1200CFD869E0E1D8D9
:1060100067E0E6D865E005019A5162E09A514008D0
:106020005FE3DF6A05019A51DF5C20E0DF50156A0B
:106030009B0F146E050E152214C0E6FF15C0E6FF77
:106040000A0EDF24DF24E76EFC0EDBCF16F0FD0E18
:10605000DBCF17F0E7501626000E172216C0E6FF1A
:1060600017C0E6FFC4D83CE0DF2ADCD7DB0EE66EC3
:10607000050EE66E0A0E9A259A253CD831E066D8C0
:10608000DB2514242DE10C0E9A259A254CD83B08CB
:1060900027E1030E48D8530A0DE0030A21E1000E60
:1060A000985D000E99591CE34BD812EC3AF057D882
:1060B00019E116D0000E985D380E995911E29A51E7
:1060C000156A9825146E99511522000ED880145423
:1060D000380E155405E334D8E0EC27F040D802E040
:1060E000000E03D04AD892D86CD8E552E552E7CFDB
:1060F000D9FF1200E76EFC0EDBCF14F0FD0EDBCFF4
:1061000015F0E7501426000E152214C0E6FF15C046
:10611000E6FFF7EF30F0FE0EDBCFE6FFA9EC34F040
:10612000E552E5521200E76EFC0EDBCFE9FFFD0EF3
:10613000DBCFEAFFE750E926000EEA22EF5012001B
:106140005ED898C5E6FF99C5E6FF120058D86EECF8
:106150004AF0E552E552E552146E06EF31F0146E46
:10616000050EE15E145000091200FE0EDBCFE6FFC3
:106170006CEC38F0E552010E1200FC0EDBCFE6FFAE
:10618000FD0EDBCFE6FFFE0EDBCFE6FF2EEC0BF0C5
:10619000E552E552E55299C5E6FFBDDF98C5E6FF39
:1061A000BADF9AC5E6FF8BEF30F0D9CFE6FFE1CF3B
:1061B000D9FFE652990EE66E050EE66E040E7AEFF2
:1061C00030F0FF0DF3CFDBF5F3CFE6FFA4DFB5EF43
:1061D00030F0980EE66E050EE66E060E7AEF30F0A1
:1061E0009A0EE66E050EE66E080E7AEF30F0D2ECEF
:1061F00035F0E552E552E552E552000912009AC524
:10620000E6FF9B0EE66E050EE66E12000501995143
:0662100098259A251200FA
:0A621600DACFE4FFE2CFDAFFE9CFB0
:10622000E4FFEACFE4FFF6CFE4FFF7CFE4FFF8CFD7
:10623000E4FFF3CFE4FFF4CFE4FFFACFE4FFFBCFBA
:10624000E4FF00EE00F0140EE80403E3EECFE4FFF9
:10625000FBD7E652CD90CECF0CFFCFCF0DFF06017E
:106260006C510F010C2706016D510F010D230DCF4D
:10627000CFFF0CCFCEFFCD809E90042B04B188D0F1
:10628000D6CF0CFFD7CF0DFFD76AD66A0CCF05FF4C
:106290000DCF06FF07014A810F010E9182AA0E81E0
:1062A000BB0E055D000E065959E30E51010B56E079
:1062B0000E51020B53E00601D50EC55D000EC65906
:1062C0004DE30F01D50E0A5D000E0B5947E30601A1
:1062D000C1510601C35D0601C2510601C4593EE227
:1062E0000F010551075D0651085906E30551075D89
:1062F0000C6F0651085905D00751055D0C6F085108
:1063000006590D6F010ED8800C55000E0D5520E377
:10631000092B0951226E236AD890235004E6060EF9
:10632000225C000E235815E3060E096F080E086E56
:10633000096A05CF0DF006CF0EF0F2EC3EF006C074
:1063400014FF07C015FF14CF12FF15CF13FF01D0A4
:10635000096B05CF07FF06CF08FF02D00F01096BBD
:106360000F010E930EB10E83C5C60AFFC6C60BFF02
:106370000F2B000E1023F40E0F5D010E105908E3D1
:106380000F6B106B002B000E0123022307014A83C1
:106390000F01115101E011070351040A57E0070AE8
:1063A0003CE0010A26E0030A12E0010A22E18250E1
:1063B000200B50E14E0E07011B5D4CE107014B51D4
:1063C00049E18B900F01020E116F010E3DD08250FA
:1063D000200B07E14E0E07011B5D03E107014B5146
:1063E00003E08B800F0135D00F01115133E18B8217
:1063F0002AD04E0E07011B5D19E107014B5116E132
:1064000082AA28D023C611FF0701395103E00F01EA
:10641000010E116F0F01030E17D0115107E04E0E40
:1064200007011B5D03E107014B5105E08B920F0152
:10643000040E116F09D08250200B0CE10701395175
:1064400009E10F01116B020E036F04D0115102E13B
:106450008B80036BE55200EE13F0140EE80403E3A7
:10646000E5CFEDFFFBD7E5CFFBFFE5CFFAFFE5CFAB
:10647000F4FFE5CFF3FFE5CFF8FFE5CFF7FFE5CF7A
:10648000F6FFE5CFEAFFE5CFE9FFE5CFDAFF110040
:0A6490008B928B800F01036B12004A
:06649A0021D9090EE126E4
:1064A00007014CA10BD0205001E181D003D9810E0E
:1064B000E66E3E0EE66E83EC2DF075D020500BE0BC
:1064C000F9D8800EE66E3E0EE66E83EC2DF0146E6B
:1064D000050EE15E14504E0E07011B5D68E1EAD81F
:1064E000C1D8E552E552E552BBEC44F0FE0EDB505C
:1064F00045085DE01F0EE66EE66AAEEC39F0E55247
:10650000E552DF6E000EFE0EDB504E0A04E01A0A62
:1065100002E0110A30E1ECD8B3EC27F0166E050E5C
:10652000E15E1650000943E1010EDB50F36EFE0EF2
:10653000DB50F35C20E1FE0EDB50540838E0D9500C
:10654000070FE96EDACFEAFFFF0EEE1802E1FF0E49
:10655000ED1811E0070EDB2A080E01E3DB2A020E1C
:1065600000CFDBFF030E01CFDBFF040E02CFDBFF0A
:10657000BFD8AED81CD0DF2A000E080EE66E1B0E68
:10658000E66E070E87D8A4D8000911E1DFCF1FF609
:10659000010EE66E1F0EE66E060EE66E1F0EE66E2E
:1065A000E66A12EC3AF0146E050EE15E1450090E24
:1065B000E15C02E2E16AE552E16E96D04E0E07011F
:1065C0001B5D09E04E0E1B6F010E216F226BBBECB1
:1065D00044F037EC45F0120007011B51490A0FE067
:1065E0001D0A12E107013E510601325D07013F51CC
:1065F000060133590AE20701030E236F1200070157
:106600004BB503D0DEEF32F0D9DF1200E66A080E98
:10661000E66EE66A380EE66E0CEC27F0E552E552BF
:10662000E552E55212005BD8AAEC2DF06AD869EC6D
:1066300038F0E552460EE66E45D84C0EE66E42D86E
:106640001BC7E6FF3FD821C7E6FF22C7E6FF59D8A0
:1066500062EC35F0E552E552E55253D86CEC38F077
:10666000E55242D03CD8FE0EDBCF1BF700CF1CF723
:1066700001CF1DF702CF1EF714CF1FF715CF20F75C
:10668000FC0EDBCF21F7FD0EDBCF22F70701080E52
:10669000236F2AD0E66EDF50080DF3CF14F0F4CF4D
:1066A00015F0000E1426380E152214C0E6FF15C092
:1066B000E6FF1200FC0EDBCFE6FFFD0EDBCFE6FFB0
:1066C00081EF33F01ED823EC38F0E552E55212008A
:1066D000E0EC27F0166E050EE15E16501200D9CFE1
:1066E000E6FFE1CFD9FF1200E552E7CFD9FF120054
:1066F000080EE66ED950010FE66E000EDA204AEF62
:0A67000033F0FE0EDBCFE6FF1200BF
:06670A000601320EF05DF5
:10671000000EF1591DE2F8C6E6FFC7D8E5520501A3
:10672000FC6FF9C6E6FFC1D8E5520501FD6F20A652
:1067300006D0FDC5E6FFFCC5E6FF1F0EEBD8050140
:10674000FF6BFE6B0601F86BF96B0601040E09D0B6
:106750000601F75105E1C9D8010EF76F060101D016
:10676000E2D8E96F120020EC42F006010C0ED8804E
:10677000F055000EF15507E206010C0ED880F555D4
:10678000000EF65503E3CFD8E96F1200070E05019E
:10679000FE5D2AE0FE2BFE51070802E2070EFE6FA7
:1067A000100EFE03F3CFF8F6FF0EFC5D14E10601B8
:1067B000F851146E156AF851A3D8E8AE02D0173418
:1067C00004D01650145C1750155803E2F851F827FE
:1067D0001200F8691200FC510601070B65E0F8434E
:1067E000F89FE806FCE11200FE6B0601F86B070E4D
:1067F0000501FF5D2DE0FF2B100EFF03F3CFF9F62F
:10680000FF0EFD5D14E10601F951146E156AF95190
:1068100077D8E8AE02D0173404D01650145C175065
:10682000155803E2F951F9270AD0F96908D0FD514A
:106830000601070B04E0F943F99FE806FCE120A6F6
:1068400033D0F9C6E6FFFFC5E6FF2B0E8AEF34F022
:106850000601F75127E149D806010E0ED880F05500
:10686000000EF1550CE307013651050808E3080E48
:106870000601EF5D04E3080E0601F95D05E206017D
:10688000010EF76F06010CD0EDC6F7F6EEC6F8F66E
:10689000EFC6F9F6F0C6FAF6F1C6FBF60601050EEC
:1068A000E96F120040D8E96F1200D9CFE6FFE1CFBF
:1068B000D9FFFE0EDB50C00B02E0FF0E12D0FE0E21
:1068C000DBAA02D0000E0DD0DBA802D0010E09D049
:1068D000DBA602D0020E05D0DBA402D0030E01D04D
:1068E000040EE552E7CFD9FF1200EDC6F2F6EEC670
:1068F000F3F6EFC6F4F6F0C6F5F6F1C6F6F61200BA
:10690000166E176AFF0ED8801656000E17561550D1
:1069100017181200E66EE66A9AEC2DF0E552E55281
:10692000E552E552120050EC42F00601050E12004D
:1069300002D9630ED8804855000E495503E2630E14
:10694000486F496BE4D851D8C8D0F5D8E0D855D8AD
:10695000C4D0C8D8FD0EDB380F0BE66EC8D809D8F6
:10696000E552E552FD0EDBCFE6FFC1D802D8E55275
:10697000B4D0B8D8FD0EDB98DB9ADB9CDB9EDB50F5
:10698000090804E2FD0EDB50370F03D0FD0EDB508B
:10699000300FE66EC8D8A1D0A5D8FD0EDB50300967
:1069A000E66EC1D89AD09ED8E652300EDF6E07014F
:1069B0004651485D4751495908E34651485F4751A0
:1069C000495BDF2A010E456FF2D7455104E0DFCF66
:1069D000E6FFA9D8E55281D085D80701010E456FA1
:1069E000466F476B84D8DFDF78D07CD80A0E07016A
:1069F000466F476B87D8F0DF70D074D8640E0701FC
:106A0000466F476B7FD8F1DF68D06CD80701E80E7E
:106A1000466F030E476F76D8F0DF5FD063D807016B
:106A2000100E466F270E476F6DD8EFDF56D05AD83D
:106A3000E150FC0FE96EFF0EDA20EA6E050EEE263D
:106A4000000EED22D950FC0FE96EFF0EDA20EA6E3F
:106A50000A0E0D6E0E6AEECF08F0EDCF09F01FECB6
:106A60004CF008C0EEFF09C0EDFF55D81CD8E55228
:106A7000E55233D037D83BD875EC38F0E5524BD8D7
:106A800026D8E552E55229D053D80701E70ED88021
:106A90004855030E495504E2E70E486F030E496F4F
:106AA00036D8ABDF1AD044D807010F0ED88048552E
:106AB000270E495504E20F0E486F270E496F27D85D
:106AC000A4DF0BD035D8070122D8A8DF06D030D8F4
:106AD0000701456B0CD8A2DF00D0E552E552E7CFA5
:106AE000D9FF1200D9CFE6FFE1CFD9FF1200FE0E89
:106AF000DBCFE6FF1200FC0EDBCF48F7FD0EDBCF4D
:106B000049F71200F4DF4FDFE55277EF35F0010E61
:106B1000456F77EF35F0FC0EDBCFE6FFFD0EDBCFE8
:106B2000E6FF77EF35F0E3DF23EC38F0E5521200B3
:106B3000D9DF7BEF35F0D6DFFD0EDB500701486F64
:046B4000496B12008B
:0C6B4400E4D8FC0EDB500FE0F1D803E3B6
:106B5000ECD8390802E2000E09D0FD0EDB2AFE0E49
:106B600001E3DB2AFC0EDB06EED7010ED5D0CFD831
:106B7000DFD816E3DAD8390813E3D2D8EFCF15F00F
:106B8000300E155C0DE3DED839080AE3DBD8D00FF0
:106B9000146ECBD8D00F0A0DF3501424ACD801D00A
:106BA000000EBAD0B4D8C4D806E3BFD8390803E37E
:106BB000BCD8D00F0CD093D8EFCF14F0410E145C9A
:106BC00014E3B3D8460811E3B0D8BF0F0A0F100D75
:106BD000F35091D8E76E83D889D894D808E3B2D817
:106BE000390805E3AFD8D00F0ED0000E13D098D8D7
:106BF000EFCF14F0410E145C0CE3A4D8460809E36F
:106C0000A1D8BF0F0A0F146E96D81450EF26010EAC
:106C100001D0000E81D07BD8040EE126DE6ADE6A48
:106C2000DE6ADD6ADD52DD5280D8200803E07DD8BF
:106C3000090806E1FD0EDB2AFE0EF6E3DB2AF4D797
:106C400077D833E372D8390830E3D9CFE9FFDACF08
:106C5000EAFF0A0E0B6E0C6A0D6A0E6AEECF06F0A2
:106C6000EECF07F0EECF08F0EFCF09F038EC4BF0A5
:106C700005C0EDFF04C0EDFF03C0EDFF02C0EFFF54
:106C800054D8D00F156A166A176AE850DE261550D8
:106C9000DE221650DE221750DD22DD52DD52FD0EBF
:106CA000DB2AFE0ECDE3DB2ACBD7D950020FE96EEB
:106CB000DACFEAFFEE50ED1003E0F368F46808D095
:106CC000DECF14F0DDCF15F014C0F3FF15C0F4FFD4
:106CD000040EE15C02E2E16AE552E16E1DD0FD0EB8
:106CE000DBCFE9FFFE0EDBCFEAFF1200E750E9261B
:106CF000000EEA221200E66E1ED8E552E750EF6E53
:106D0000010E1200EFCF14F0300E145C1200D9CF38
:106D1000E6FFE1CFD9FF1200E552E7CFD9FF12001D
:106D2000010EE76EDCDF76EF36F0D9DFEF501200B0
:106D3000D6DF82EF36F0FB0EDBCFE9FFFC0EDBCFB8
:0A6D4000EAFF1200EDDFEF50120031
:066D4A007FEC4BF070EC41
:106D50004BF0D08EF28CF28E35EC0FF00701556BB4
:106D600088EC39F050EC44F0E7EC1AF0CBEC43F04F
:106D700048EC32F0F7EC4AF0FCEC4AF007010F0E59
:106D8000366F0A0EE66E92EC1FF0E55294EC27F097
:106D9000000908E1010EE66EE66A4E0EE66E4DEC65
:106DA00032F007D0010EE66EE66A450EE66E32EC72
:106DB00033F0E552E552E55284EC4CF0D18002EC20
:106DC00038F0E1EF37F007014AA136D04A910701C8
:106DD0005E2B0701625104E0620702E1D3EC0EF082
:106DE00007015EB11ED082BA02D007014D8B070E9B
:106DF00007015E1510E107014D8B07014CAB02D076
:106E000007014D8307014D854D891F0E07015E1552
:106E100002E107014D8107014DAB0ED0E7EC1EF0FA
:106E20000BD01AEC2AF007014AA304D04A930701B9
:106E30004D8D0CD8ADEC46F00701625102E1CEEC6D
:106E40000FF022EC46F0EAEC48F0BDD700016051AB
:106E500001E060070701105101E010070601FC5135
:106E600011E0D6EC28F000090DE10601FC070AE16B
:106E700020AC08D0920EE66E010EE66E06EC2DF008
:106E8000E552E5520701635122E06351146E156A21
:106E9000FF0E141801E115501AE0560E0701695D46
:106EA0000DE10601DE51DF1109E107011E0E4E5D05
:106EB000000E4F5903E20701636B09D038EC0FF065
:106EC000000903E025C663F702D007016307070145
:106ED00063510EE107014C51040B0AE00601DE513B
:106EE000DF1106E138EC0FF0000902E10DEC41F092
:106EF0000701235104E0230702E1ECEC32F0060124
:106F000036510601CF5D060137510601D05903E322
:106F100007015F6B10D007015F2B030E5F5D0BE372
:106F2000CFC6E6FFD0C6E6FF4C0EE66E4DEC32F063
:0A6F3000E552E552E55284EF4CF003
:066F3A004F0EAB169D9AFC
:106F4000AC9A9D9812004F0E0F012217A39A219B15
:106F5000A3981200D4D8E65207010151005DFCE06D
:106F60000051002BEA6A0225E96E0351CDD0C7D843
:106F7000E65207010551045DFCE00451042BEA6A66
:106F80000625E96E0751C0D007010151005D01E1FE
:106F9000000C010C07010551045D01E1000C010C1E
:106FA00007010951085D01E0010CACA2010C000CC5
:106FB00007010D510C5D01E0010C0F0121A3010C33
:106FC000000CBBDF0701086B096B000E0A6F020E95
:106FD0000B6F656A27C6AFFF450EAC6E9F98AC8AF3
:106FE000006B016B000E026F040E036F100EAB6E90
:106FF0009F9AAB8EAE50E86EAE50E86EAE50E86E23
:107000009D8A1200A0DF07010C6B0D6B000E0E6F46
:10701000010E0F6F0F01206B28C61EFF450E216F5A
:10702000A598218B0701046B056B000E066F030EFC
:10703000076F0F01100E226FA59A228F1D511D514F
:107040001D51A38A12005BD8FE0EDB50010A07E037
:10705000010A0AE1FD0EDBCFE6FF0AD804D0FD0EDF
:10706000DBCFE6FF1DD8E552E552E7CFD9FF12008E
:1070700046D8E652ACAA13D009C7DFFFDF2A0701C2
:107080000851DF5CFCE00951EA6A0A25E96E0B5100
:10709000EA22FE0EDBCFEFFFDFCF09F79D8839D064
:1070A0002ED8E6520F0121AB13D00DC7DFFFDF2A28
:1070B00007010C51DF5CFCE00D51EA6A0E25E96E18
:1070C0000F51EA22FE0EDBCFEFFFDFCF0DF7A388D3
:1070D00020D015D85E0E11D012D83B0E0ED00FD88E
:1070E0000D0E1CD8E5520A0E08D009D8200E05D086
:1070F000200EE66EBDDFE552120010D80AD0D9CFBF
:10710000E6FFE1CFD9FF1200EA22EFCFDFFFDF5029
:1071100000D0E552E552E7CFD9FF1200E66EFE0E31
:0A712000DBCFE6FF90DFE55212001E
:06712A00D9CFE6FFE1CF22
:10713000D9FF060EE126D950FB0FE96EFF0EDA20CB
:10714000EA6EEE50ED1075E0DCD8D4D81450165C21
:10715000155017585EE2CED8FD0EDB501624146E83
:10716000FE0EDB501720156E000E14C0DFFF010E5F
:1071700015C0DBFF020EDB6A030EDB6AB6D80A0E0F
:107180000B6E0C6A0D6A0E6AA7D838EC4BF005C07E
:10719000EDFF04C0EDFF03C0EDFF02C0EFFFFD0EE9
:1071A000DBCF16F0FE0EDBCF17F0FB0EDB50165CCC
:1071B000146EFC0EDB501758156E040E14C0DBFF66
:1071C000050E15C0DBFF040EDBCF14F0050EDBCF80
:1071D00015F0166A176A89D814C00BF015C00CF0A8
:1071E00016C00DF017C00EF077D8CBEC4BF009C0ED
:1071F000EDFF08C0EDFF07C0EDFF06C0EFFF75D83B
:10720000E70EEE5C030EEE58000EEE58000EEE5840
:1072100005E3E70EF36E030EF46E18D066D8D8803F
:107220000A0EEE54000EEE54000EEE54000EEE5414
:1072300004E30A0EF36EF46A09D0DFCF14F0010EF6
:10724000DBCF15F014C0F3FF15C0F4FF060EE15CB0
:1072500002E2E16AE552E16EE552E7CFD9FF1200A2
:10726000060E215C17E1020E0601E95D13E306013B
:10727000F0510601F55D0601F1510601F65905E2EE
:10728000F5C6F3FFF6C6F4FF1200F0C6F3FFF1C631
:10729000F4FF12004EC7F3FF4FC7F4FF1200D9CF1F
:1072A000E6FFE1CFD9FF2DD80A0E145C000E155869
:1072B0000CE3D950FD0FE96EFF0EDA20EA6EE70EFF
:1072C000D880EE54030EED5402E2000E01D0010E00
:1072D000E552E7CFD9FF1200EECF06F0EECF07F070
:1072E000EECF08F0EFCF09F01200D9CFE9FFDACFE7
:1072F000EAFF1200FB0EDBCF16F0FC0EDBCF17F01F
:107300001200FD0EDBCF14F0FE0EDBCF15F01200E5
:107310007F94A698A99860881200B0D802E3000E66
:1073200001D0010EB7D0AAD802E3000E16D0FC0E91
:10733000DBCF14F0FD0EDBCF15F0FE0EDBCF16F029
:10734000000ED8801556040E16561450155C000E0B
:10735000165802E3010E01D0000E9CD0D9CFE6FFF3
:10736000E1CFD9FF17D8FD0EDBCF14F0FE0EDBCF37
:1073700015F015C014F0156A1450636EFD0EDB5045
:10738000626E7F6A7F800000615000D0E552E7CFD7
:10739000D9FF12007FB2FED77F94120094D8FADF93
:1073A00066D8BBDFE552E552000902E1000E18D0B5
:1073B000FE0EDBCF15F015C014F0156A1450636E85
:1073C000FD0EDB50626EFC0EDB50616E7F6A7F84C7
:1073D000F29E550E7E6EAA0E7E6E7F82F28E010E9A
:1073E00059D071D875D802E1000E1BD065D818E0CD
:1073F000FD0EDBCF14F0DB2AFE0EDBCF15F001E330
:10740000DB2A14C0E6FF15C0E6FFA8DFE552E5520F
:10741000E66E44D801E3DB2AE552E750EF6EE6D78B
:10742000010E38D050D8E65253D802E1000E1DD0DC
:1074300043D81AE033D801E3DB2AEFCFDFFF17D8B8
:107440008DDFE552E552146EDF50145C07E0DFCFAC
:10745000E6FF0DD8A3DFE552E552E552FD0EDB2A2B
:10746000FE0EE6E3DB2AE4D7010EE55213D0FD0E53
:10747000DBCFE6FFFE0EDBCFE6FF120024D8FD0EC9
:10748000DBCF14F0FE0EDBCF15F0000E145C040E03
:1074900015581200E552E7CFD9FF1200FB0EDBCFE3
:1074A000E9FFDB2AFC0EDBCFEAFF12003CDFE552EE
:1074B000E552E55200091200FA0EDBCFF3FFDB06BE
:1074C000F35000091200D9CFE6FFE1CFD9FF120037
:0C74D000FA0EDBCFE6FFCBDF56EF3AF000
:0474DC00C5D8AAEC79
:1074E0002DF094D8540EBDD823EC38F0E552E55277
:1074F000530EB7D823EC38F0ADD82150B2D8CCEC2D
:1075000034F0A8D8E9C6E6FFC5D8CCEC34F0A2D850
:10751000EAC6E6FFEBC6E6FFBDD844EC35F0E5521F
:1075200099D84EC7E6FF4FC7E6FFB4D844EC35F014
:10753000E552E552E552AED86CEC38F0E55299D000
:10754000205020E0AAEC2DF0410E97D8550E95D88A
:10755000540E93D84F0E91D878EC38F014CFE6FF44
:1075600015CFE6FFE66A62EC35F0E552E552E552EA
:1075700078EC38F04EC7E6FF4FC7E6FFE66A44EC0A
:1075800035F080D8120070D8205004E0AAEC2DF01D
:10759000460E54D86ED068D8205004E0AAEC2DF0E6
:1075A0004D0E4CD866D020A630D00601EA51070116
:1075B00042191AE10601EB510701431915E1215067
:1075C000405D12E10601E9510701415D0DE14451C1
:1075D000146E156AD890155004E6E70E145C030E7D
:1075E000155802E2442B1200AAEC2DF021C040F7FE
:1075F000E9C641F7EAC642F7EBC643F7E66A6FEC25
:1076000038F0E552E66A6ADFE5521200070144519C
:1076100014E0540E32D8530E30D8520E2ED8070133
:107620004451E66EE66AE66A3AEC35F02BD807017B
:10763000446B406B416B426B436B12001ED8540E7F
:107640001CD8FD0EDBCFE6FF25D8E66A62EC35F0EC
:1076500042EF3BF0E552E5521DD875EC38F0E552AB
:107660001200E66E4AEF3BF0D9CFE6FFE1CFD9FF3B
:107670001200E552E7CFD9FF1200E66E38EC38F081
:10768000E5521200E552E552E552E66A6CEC38F03C
:0C769000E5521200FE0EDBCFE6FF1200F8
:04769C000601E70EEE
:1076A000F06F030EF16FAAD80701526F080EBAD817
:1076B00002E0BCD8FEE10601EF6F0601F96F800E13
:1076C000B1D802E0B3D8FEE10701536F010E546F49
:1076D000100EA8D802E0AAD8FEE10601EE6F06015E
:1076E000F86F0601020EE96F1200D9CFE6FFE1CF75
:1076F000D9FFE65220EC42F006010E0ED880FA5572
:10770000000EFB5517E3EDC6F7F6EEC6F8F6EFC62A
:10771000F9F6F0C6FAF6F1C6FBF60601030EE96FBC
:1077200006010C0ED880FA55000EFB5547E3060102
:10773000050E43D00F0E0701545D10E2542B0601D5
:10774000FC510AE00701542B0601E70EFA5D030E17
:10775000FB5902E30701542B36D830D0010E546F89
:1077600032D8070153510601F95D21E2F9C6DFFF66
:107770000601FC510FE0010EDF6E020E0701365DBF
:1077800001E2DF2A0601E70EFA5D030EFB5902E370
:10779000DF50DF260601F9510701535DDF5C04E28B
:1077A000DF500601F9270AD053C7F9F607D0EEC615
:1077B000F8F6EFC6F9F60601030EE96FE552E55259
:1077C000E7CFD9FF1200100E0701545D0AE2100E38
:1077D0005403F35027D802E029D8FEE10601F86FE0
:1077E0001200FF0E1FD802E021D8FEE10601F86F5B
:1077F0000701525102E00601F82B12000701365131
:10780000050A0EE0030A0CE0050A09E0070A07E092
:10781000040A04E0010A02E0030A03E1000C010C7F
:10782000020C030C52C7E7FFE7521200E8427F0B3D
:04783000E706120055
:0C783400D8CFE4FFE0CFE4FFE46EDACF31
:10784000E4FFE9CFE4FFEACFE4FFE6529DAA42D08D
:107850009EAA40D0ABA203D0AB98AB88F9D7ABA41B
:1078600002D0AE50F5D7070110511FE00F01215192
:10787000200B1BE007010D51EA6A0E25E96E0F513E
:10788000EA22AECFEFFF0DC765F70701652B655103
:1078900007010C5D02E065C70DF7A388050E07011F
:1078A000105DD6E2050E106FD3D707010151EA6AC9
:1078B0000225E96E0351EA22AECFEFFF01C765F75B
:1078C0000701652B070100510701655DC1E065C730
:1078D00001F7BED7A3AA3CD0A4AA3AD00F0122A395
:1078E00003D022992289F8D722A502D01D51F4D7BE
:1078F0000701105119E0AC50200B16E007010951A7
:10790000EA6A0A25E96E0B51EA221DCFEFFF09C78B
:1079100065F70701652B070108510701655D02E066
:1079200065C709F79D88D8D707010551EA6A06257A
:10793000E96E0751EA221DCFEFFF05C765F7070182
:10794000652B65510701045DC7E065C705F7C4D71E
:107950009D50100B12E09E50100B0FE007010851D4
:10796000095D02E19D9809D00851EA6A0A25E96E8D
:107970000B51EA22EF50AD6E082BA350100B13E011
:10798000A450100B10E007010C510D5D02E1A3980B
:10799000F4D70C51EA6A0E25E96E0F51EA22EFCFB7
:1079A0001CFF0C2BEAD7A6A802D0A6987F94E5521C
:1079B000E5CFEAFFE5CFE9FFE5CFDAFFE550E5CF18
:0879C000E0FFE5CFD8FF100045
:0879C800D9CFE6FFE1CFD9FFA2
:1079D000200EE126D9CFE9FFDACFEAFFDCC5EEFFC2
:1079E000DDC5EEFFDEC5EEFFDFC5EEFFE0C5EEFF55
:1079F000E1C5EEFFE2C5EEFFE3C5EEFFE4C5EEFF35
:107A0000E5C5EEFFE6C5EEFFE7C5EEFFE8C5EEFF14
:107A1000E9C5EEFFEAC5EEFFEBC5EEFFECC5EEFFF4
:107A2000EDC5EEFFEEC5EEFFEFC5EEFFF0C5EEFFD4
:107A3000F1C5EEFFF2C5EEFFF3C5EEFFF4C5EEFFB4
:107A4000F5C5EEFFF6C5EEFFF7C5EEFFF8C5EEFF94
:107A5000F9C5EEFFFAC5EEFFFBC5EEFFFD0EDB50EC
:107A60000701365D0EE0FD0EDBCFE6FFD9CFE6FF66
:107A7000DACFE6FFF7EC1AF0E552E552E5520009DD
:107A80002DE048D869EC38F0E552540E3CD8420E4F
:107A90003AD8FD0E34D898EC34F02AD8040EDBCF57
:107AA000E6FF050E2CD8C7EC4AF0E55221D8060EA9
:107AB000DBCFE6FF070EDBCFE6FF080E20D8AEECEB
:107AC00017F0E552E55214D8090E19D8A0EC47F08A
:107AD000E552E5521FD86CEC38F0E552200EE15C1F
:107AE00002E2E16AE552E16EE552E7CFD9FF12000A
:107AF000E552E5520FD875EC38F0E5521200DBCFB5
:107B0000E6FF8AEF3DF0E66E05D823EC38F0E5524B
:0C7B1000E5521200FE0EDBCFE6FF120073
:047B1C00500EE66EB3
:107B2000E66AE668300EE66E060E90D80601580E3C
:107B3000306F020E316F260E326F020E336FF00E71
:107B4000346F356B280E366F230E376F800E386F0B
:107B50003E0E396F200E3A6F030E3B6F400E3C6FA6
:107B6000060E3D6F3CC63EF63DC63FF6B00E406F7A
:107B7000360E416FD00E426F070E436F700E446F8A
:107B8000170E456F700E466F170E476F200E486F29
:107B90004E0E496F190E4A6F4B6B640E4C6F4D6B56
:107BA000190E4E6F4F6BC40E506F090E516F880E39
:107BB000546F130E556F120E606F616B0A0E626F79
:107BC000636B0C0E646F656B1E0E666F676BB40E95
:107BD000686F696B040E6A6F6B6B6B0E6C6FF00EE7
:107BE0006D6F500EE66E300EE66E060EE66E300ECF
:107BF00024D0100EE66EE66AE668200EE66E060EEB
:107C000025D80601AA0E206F080E216F100E226FD4
:107C1000236B030E246F080E256F190E276F286F34
:107C2000440E296F4D0E2A6F2B6B100EE66E200E40
:107C3000E66E060EE66E200E00D0E66EE66A12ECE8
:107C40003AF0146E050EE15E14501200E66EEFEC91
:0C7C50004BF0146E050EE15E14501200A3
:047C5C000601EA2B08
:107C6000000EEB2372EC42F020A602D0EDEC49F0BE
:107C70000601FA510601625D0601FB5106016359D6
:107C800003E30601EC8125D00601E951060A1FE055
:107C90000F0A1DE00C0A18E0010A13E0070A0EE0C3
:107CA000010A09E0030A04E0010A13E12ED811D009
:107CB0004EEC3BF00ED075EC3BF00BD085EC33F086
:107CC00008D0B3EC33F005D095EC2BF002D0F7ECF4
:107CD0002BF09EEC42F00601ECA116D020EC42F015
:107CE0000601FA510601665D0601FB51060167595E
:107CF0000BE2FAC6E6FFFBC6E6FF410EE66E4DEC70
:107D000032F0E552E552E55212000601E70EF56F3A
:107D1000030EF66F0E0ED880FA55000EFB5521E3C8
:107D2000F7C6EDF6F8C6EEF6F9C6EFF6FAC6F0F6C7
:107D3000FBC6F1F6F7510AE1EDC6F2F6EEC6F3F630
:107D4000EFC6F4F6F0C6F5F6F1C6F6F6030EE96FE7
:107D50000C0ED880FA55000EFB5506E3050EE96FB0
:107D60001200F76B010EE96F12000601E96BEA6B76
:107D7000EB6BEC6BE70EF56F030EF66FF5C6F0F6E6
:0A7D8000F16FF5C6FAF6FB6F120072
:067D8A0009C013F008C05F
:107D900012F008500D02F4CF07F0F3CF06F00950AF
:107DA0000E02F4CF09F0F3CF08F00D02F3500726CE
:107DB000F4500822E86A092212500E02F3500726F6
:107DC000F4500822E86A09220EAEEBEF3EF01250A2
:107DD000085E1350095A13AE000C0D50085E0E5089
:107DE000095A000C08C012F008500D02F4CF07F039
:107DF000F3CF06F009500E02F4CF09F0F3CF08F0EC
:107E00000D02F3500726F4500822E86A09221250A6
:107E10000E02F3500726F4500822E86A0922000CEB
:107E200009C013F008C012F007C011F007500C028F
:107E3000F4CF05F0F3CF04F008500D02F4CF07F0B3
:107E4000F3CF06F00C02F3500526F4500622E86A40
:107E5000072211500D02F3500526F4500622E86A5D
:107E6000072209500C02F3500626F450072209504D
:107E70000D02086AE86A0822F3500726F450082227
:107E800011500E02F3500626F4500722096AE86AE0
:107E90000822092212500E02F3500726F45008223D
:107EA000E86A092213500E02F3500826F450092202
:027EB000000CC4
:0E7EB20086D87ED8EF50800B05E0E5EC47F057
:107EC000000905E024D0E5EC47F0000920E071D876
:107ED000EF50400B05E042EC48F0010805E017D0F8
:107EE00042EC48F0000913E131EC43F0146E61D824
:107EF000EE52EF50145C0BE1ABEC42F0146E59D82B
:107F0000020EE926000EEA22EF50145C02E0000E99
:107F100001D0010E5AD054D8030EE126DF6AD9CF22
:107F2000E9FFDACFEAFF8F50080B02E0EF8E01D0B5
:107F3000EF9E42EC48F0010801E1DF8C31EC43F0A8
:107F4000E76E010EE7CFDBFFABEC42F0E76E020E0F
:107F5000E7CFDBFFDFCF14F0010EDBCF15F0020E11
:107F6000DBCF16F014C007F015C008F016C009F0FA
:107F7000030EE15C02E2E16AE552E16E26D020D810
:107F8000F90EDB50F36EFC0EDB50F35C0EE1FA0EE3
:107F9000DB50F36EFD0EDB50F35C07E1FB0EDB50B4
:107FA000F36EFE0EDB50F35C02E0000E01D0010E1A
:107FB0000CD0FD0EDBCFE9FFFE0EDBCFEAFF120097
:107FC000D9CFE6FFE1CFD9FF1200E552E7CFD9FFC5
:027FD00012009D
:0E7FD200090E216E38EC0FF000090DE120AA17
:107FE00023D04EC6E6FF4FC6E6FFD8C6E6FFD9C689
:107FF000E6FFE40E67EF40F018EC29F0000901E11C
:10800000120020A60AD060C6E6FF61C6E6FF4EC792
:10801000E6FF4FC7E6FFF80E5AD807014C9D000156
:10802000FA89FA83040E216E120077EC45F00009FC
:1080300008E020A602D0100E42D80F01035101E043
:108040001200E5C5E6FF68EC29F0E552000904E0FE
:1080500020AE34D02E0E19D0A6EC41F0420804E038
:108060000501E251800B09E1580EE66E070E39D882
:108070000EE020AE23D0380E08D0E20EE66E050EDC
:1080800030D805E020A61AD0390E5FEF40F000018D
:10809000FAA906D020A602D0420E11D8040E0AD0AA
:1080A00006014E510601D85D06014F510601D9590E
:1080B00003E3020E216E1200090E216E1200E66E1D
:1080C000040EE66E06EC2DF0E552E5521200E66E67
:1080D000070EE66E1CEC2DF0146E060EE15E1450D9
:1080E0001200E66EB4EC29F0E552E55200091200E8
:1080F00022D80D0A1EE0010A1BE0030A18E0010A5B
:1081000015E0070A12E00E0A0FE0010A0CE0030A6C
:1081100009E0010A06E00E0A03E0010A0BE1000C87
:10812000010C020C030C040C050C060C070C080CCB
:10813000090C0A0C0F0C62D8E652DF6A90BCDF868D
:1081400090BEDF848EB4DF828EB6DF80DF50E552D2
:108150005AD054D8FE0EDB500A0A28E0030A24E065
:10816000010A20E00F0A1CE0010A18E0030A14E0EB
:10817000010A10E0070A0CE0010A08E0030A04E023
:10818000010A16E10B0E15D00A0E13D0040E11D001
:10819000050E0FD0060E0DD0070E0BD0090E09D01C
:1081A0000E0E07D00F0E05D00C0E03D00D0E01D011
:1081B000000E29D023D8E652FE0EDBCFE6FFC9DF42
:1081C000E552DF6EDF500701645D16E0DFCF64F734
:1081D00064A702D0908C01D0909C64A502D0908EB0
:1081E00001D0909E64A302D08E8401D08E9464A1AD
:1081F00002D08E8601D08E96E55205D0D9CFE6FF0B
:0E820000E1CFD9FF1200E552E7CFD9FF1200FF
:02820E0081D815
:1082100001E1155001E0636B120007014C9599BA1A
:10822000000C908A998A0701050E626F205003E0C6
:10823000E66A4BD8E552010CD9CFE6FFE1CFD9FF72
:1082400007014B51040B1AE18750200B17E024D88B
:1082500007014C85FE0EDBCF69F720500FE00601C9
:108260002551E66EE66A5CD8AE0EE66E9C0EE66EB2
:1082700083EC2DF0146E050EE15E145007014C5195
:10828000040B06E046D801E1155002E025C663F76D
:10829000E552E7CFD9FF120007014C9587AA000CE1
:1082A000909A999A0701050E626F205003E0E66AE2
:1082B0000CD8E552010C9950200B04E18750200B9B
:1082C00001E1010C87AA020C000CD9CFE6FFE1CF37
:1082D000D9FFAAEC2DF024D869EC38F0E552410E14
:1082E00011D8540E0FD8E7DFE66E1AD8CCEC34F074
:1082F000E552E55215D86CEC38F0E552E552E7CF7F
:10830000D9FF1200E66E0CD823EC38F0E552E552A6
:10831000120007016351146E156AFF0E1418120043
:08832000FE0EDBCFE6FF1200A8
:0883280006012A51420A09E096
:108330000F0A05E00C0A01E01200420E03D0410EC4
:1083400001D04D0EE66E37D8E552120006012A51D3
:10835000120007014CAB000CF9DF410801E1010CF0
:10836000F5DF4D0801E1010C000C61D8FE0EDB5079
:10837000410A04E0030A02E00F0A02E1010E01D003
:10838000000E5AD054D8AAEC2DF0FE0EDBCFE6FF3B
:1083900069EC38F0E5524D0EE66E41D8440EE66EBB
:1083A0003ED82AC6E6FF3BD8FE0EDBCFE6FF6CECDC
:1083B00038F0E55241D03BD8E6522AC6DFFFFE0E28
:1083C000DB5006012A5D07E0FE0EDBCFE6FFCDDFC6
:1083D000E552000902E1000E20D0FE0EDBCF2AF6A6
:1083E000010EE66E2A0EE66E060EE66E2A0EE66EAA
:1083F000E66A12EC3AF0146E050EE15E145020505D
:1084000003E0E66ABFDFE552420EDF5C05E1A1DF73
:10841000000902E00001FA8B010EE5520DD0FE0EBC
:10842000DBCFE6FF23EC38F0E552E5521200D9CF5E
:10843000E6FFE1CFD9FF1200E552E7CFD9FF1200E6
:108440000601F0510601FA5D0601F1510601FB59E2
:1084500023E2F7C6EDF6F8C6EEF6F9C6EFF6FAC671
:10846000F0F6FBC6F1F6F75113E10601F5510601EE
:10847000FA5D0601F6510601FB590AE2EDC6F2F675
:10848000EEC6F3F6EFC6F4F6F0C6F5F6F1C6F6F66C
:1084900020A602D014EC4AF0120024D820EF42F0BB
:1084A0000601F5510601F05D0601F6510601F1598C
:1084B0000AE3F2C6EDF6F3C6EEF6F4C6EFF6F5C63D
:1084C000F0F6F6C6F1F6EDC6F7F6EEC6F8F6EFC62C
:1084D000F9F6F0C6FAF6F1C6FBF620A602D00DECCE
:1084E0004AF012000601E70EFA6F030EFB6F060159
:1084F0004C510601D85D06014D510601D9590EE3D4
:108500004EC7E6FF4FC7E6FF4FEC39F0E552E552A4
:10851000000904E04EC7FAF64FC7FBF642EC48F0FC
:108520000601F76F31EC43F00601F86FABEC42F057
:108530000601F96F1200B4DF9EEF42F00601F70565
:1085400003E10501E28D02D00501E29DF8C6E3F5E5
:06855000F9C6E4F512007B
:0A85560077D8E652DF6A91B8DF8E95
:108560008CBADF8C8FB0DF8A8CB8DF888CB6DF8660
:108570008DB0DF8490B4DF828CB4DF80DF505ED0BA
:1085800062D8AAEC2DF069D869EC38F0E55260D8D1
:1085900006D8E552E55261D86CEC38F04FD053D88C
:1085A0004C0E45D8520E43D853D8A9EC34F0E552BE
:1085B00045D049D8D0DF146EFE0EDB50145C02E1CA
:1085C000000E31D0FE0EDBAE02D0918801D0919822
:1085D000DBAC02D08C8A01D08C9ADBAA02D08F80CF
:1085E00001D08F90DBA802D08C8801D08C98DBA6BC
:1085F00002D08C8601D08C96DBA402D08D8001D075
:108600008D90DBA202D0908401D09094DBA002D0A8
:108610008C8401D08C94205005E01FD8E66AB0DF2E
:10862000E552E552010EE552E7CFD9FF1200E66EA2
:1086300014D823EC38F0E552E5521200E552E55229
:10864000E7CFD9FF1200D9CFE6FFE1CFD9FF120063
:10865000FD0EDBCFE6FF2DEF43F0FE0EDBCFE6FF96
:02866000120006
:0E86620077D8E652DF6A8EBADF8E8DB2DF8CDB
:108670008EBCDF8A8DBEDF888EBEDF868BB4DF8442
:108680008FB8DF8291BEDF80DF505ED062D8AAEC67
:108690002DF069D869EC38F0E55260D806D8E5527B
:1086A000E55261D86CEC38F04FD053D8430E45D822
:1086B000520E43D853D8A9EC34F0E55245D049D8EE
:1086C000D0DF146EFE0EDB50145C02E1000E31D0E0
:1086D000FE0EDBAE02D08E8A01D08E9ADBAC02D0C9
:1086E0008D8201D08D92DBAA02D08E8C01D08E9C1F
:1086F000DBA802D08D8E01D08D9EDBA602D08E8E9F
:1087000001D08E9EDBA402D08B8401D08B94DBA29F
:1087100002D08F8801D08F98DBA002D0918E01D03B
:10872000919E205005E01FD8E66AB0DFE552E55281
:10873000010EE552E7CFD9FF1200E66E14D823EC04
:1087400038F0E552E5521200E552E552E7CFD9FF85
:108750001200D9CFE6FFE1CFD9FF1200FD0EDBCF2B
:0E876000E6FFB3EF43F0FE0EDBCFE6FF1200A4
:02876E00C59AAA
:10877000C588C5B8FED71200C750040B01E0010E32
:10878000146E1F0EC5141410F7E11200C58AC588B7
:10879000C5B8FED712003F0EC716C66AC56AC686A0
:1087A000C78E94869488C68A270EC86E1200C58626
:1087B000C7A0FED7C9501200C582C5B2FED71200AD
:1087C000C580C5B0FED71200C584C5B4FED712005F
:1087D0004AD8FE0EDB50C96EC6AE02D0FF0E08D0DE
:1087E000C7B0FED7C9DFC5AC02D0FE0E01D0000E67
:1087F0003FD039D831D813E0DADFE66E25D801E36F
:10880000DB2AE552E750EF6EC5B6FED7A1A602D02F
:10881000FF0E06D0FC0EDB50EDE0A9DFEBD7000E1B
:1088200027D021D8E65218D80CE00ED801E3DB2A75
:10883000EF50E66ECDDFE552DF6EDF50F4E0DF5043
:1088400001D0000EE55214D0FD0EDBCFE9FFDB2A8C
:10885000FE0EDBCFEAFF1200FC0EDBCFF3FFDB06E0
:10886000F35000091200D9CFE6FFE1CFD9FF120083
:08887000E552E7CFD9FF120029
:088878000601026903691A0EF2
:10888000E66EE66AE668060EE66E060EE66EEFEC4B
:108890004BF06CD8200E5AD812EC3AF0B6EF44F0F8
:1088A000800E54D8F1EC39F061D828D8000902E1E3
:1088B000F9EC3DF08EEF3DF052D8410A08E0050A90
:1088C00006E00D0A04E0110A02E0010A02E1010ECD
:1088D00001D0000EE552E7CFD9FF120040D8190AA7
:1088E00006E02A0A04E0540A02E0A80A02E1010EA6
:1088F00001D0000EE552E7CFD9FF1200AA0E060103
:10890000205D01E0000C080E215D01E0000C225109
:10891000146E156A100E141801E1155001E0000CD8
:1089200027C6E6FFDBDFE552000901E1000C28C69F
:10893000E6FFD4DFE552000901E1000C29C6E6FF9D
:10894000BBDFE552000901E1000C010CE66E000EF0
:10895000E66E060EE66E000EE66EE66A1200D9CFEF
:10896000E6FFE1CFD9FFFE0EDB501200146E050EBC
:06897000E15E145012004C
:0A897600D9CFE6FFE1CFD9FFE652AA
:108980009050100B01E0010EDF6E07014BB521D0B6
:10899000490E07011B5D09E00601DC5106013E5D41
:1089A0000601DD5106013F5916E220AA12D03EC64B
:1089B000E6FF3FC6E6FFDCC6E6FFDDC6E6FFB30E18
:1089C000E66E9C0EE66E1CEC2DF0146E060EE15E5B
:1089D0001450909801D0908820501AE09050100BBD
:1089E00001E0010EDF5C14E0500E3CD8410E3AD895
:1089F000420E38D89050100B01E0010EE66EE66A88
:108A0000CCEC34F0E552E552E66A6CEC38F0E55215
:108A1000E552E552E7CFD9FF120007014B95BBEFB6
:108A200044F007014B85BBEF44F007016751400A52
:108A300018E0700A16E0100A0DE0300A05E0100A8E
:108A400001E01200100E04D007014B950701200E23
:108A5000676F120007014BA502D011EF45F00DEF33
:0E8A600045F01200E66E38EC38F0E5521200D8
:028A6E000701FE
:108A70004BA3000C4E0E07011B5D01E0000C90A8FB
:108A80002ED087BA16D00601DC5106013C5D0601E6
:108A9000DD5106013D5923E220AA0AD03CC6E6FF7B
:108AA0003DC6E6FFDCC6E6FFDDC6E6FF2D0E4DD86F
:108AB000000C0601DC5106013A5D0601DD5106019C
:108AC0003B590DE220AA0AD03AC6E6FF3BC6E6FFB4
:108AD000DCC6E6FFDDC6E6FF2E0E37D8000C070128
:108AE0004B93205003E0E66A0CD8E552010C0701D5
:108AF0004BB3000C4B83205003E0E66A02D8E552EA
:108B0000010CD9CFE6FFE1CFD9FFAAEC2DF04B0E37
:108B100013D8490E11D807014BA302D0310E01D052
:108B2000300E0AD8FE0EDBCFE6FF6CEC38F0E552D3
:108B3000E552E7CFD9FF1200E66EFE0EDBCFE6FF6F
:108B400023EC38F0E552E5521200E66E010EE66EB7
:0A8B50001CEC2DF0060EE15E120091
:068B5A000001FAAD0FD08E
:108B6000FA9DFDC0E6FF69EC38F0E552460E5AD892
:108B7000450E58D8FDC0E6FF6CEC38F0E552A6EC87
:108B800041F0420804E00501E251800B0FE1580E6C
:108B9000E66E070EE66EB4EC29F0E552E5520009E8
:108BA00005E020A639D0780E1AEF46F037EC45F0F4
:108BB0000001FA51100B03E1FA51020B27E020A645
:108BC00022D0F00E37D8450E28D84E0E26D8440EA7
:108BD00024D8540E22D8550E20D84E0E1ED8450E3D
:108BE0001CD878EC38F014CFE6FF15CFE6FFE66A24
:108BF000B3EC4AF0E552E552E552E66A8AEC49F0F8
:108C0000E55266EC18F00601050EFC6F0001FA6BE8
:108C1000FB6B216AD3EC0EF01200E66E38EC38F0F4
:108C2000E5521200E66EFDC0E6FF23EC38F0E55297
:108C3000E5521200E66E230EE66E06EC2DF0E552CC
:048C4000E5521200E7
:0C8C4400C4EC37F000096DE0AAEC37F03A
:108C50000501976FE85002E100510CE00051EA6A0B
:108C6000010FE96E050EEA2297C5EFFF960E005D33
:108C700001E2002B3B0E975DE5E101515E0A0EE03B
:108C8000650A08E0580E0601295D1EE0440E295DC4
:108C900047E11AD0E66A6CEC38F014D000C5E6FF64
:108CA000010EE66E050EE66E23EC4AF0E552E55243
:108CB000E552010EE66E050EE66EE66A8AEC20F0DD
:108CC000E552E552E5522CD00501006B0051002B16
:108CD000EA6A010FE96E050EEA22EFCF97F597C514
:108CE000E6FF50EC38F0E5523B0E0501975DEEE1F2
:108CF0004C0E015D15E1440E025D12E1460E035D6E
:108D000009E1320E045D06E13B0E055D03E107015A
:108D10001E0E05D0050E0701105D02E2050E106F54
:088D20000501006B8FD7120062
:088D2800215016E0090A14E0D5
:108D3000205010E0090EE66EE66A2150E66EE66A03
:108D4000880EE66E130EE66E1CEC2DF0146E060E09
:108D5000E15E1450090E216E12000001F95102E08B
:108D6000F9071200020EF96F2150090A46E00F0AB6
:108D700031E0030A25E0010A1CE0060A13E0030AB9
:108D80000AE0010A01E01200FAEC23F0215038E178
:108D90000001F96B1200C1EC28F0000915E131D88F
:108DA00015EF40F0C1EC28F000090EE12AD8E9EFF8
:108DB0003FF0C1EC28F0000907E123D884EF2EF042
:108DC000C1EC28F0000903E0090E216E120019D849
:108DD00067EF2EF016D822EC2FF00601ECA110D090
:108DE00020AC07D02F0EE66EE66A06EC2DF0E552B9
:108DF000E55200010C0EF96F120003D8ADEF45F0FB
:0A8E00001200C6EC11F0D3EF3AF0B7
:068E0A0045D800090FE04D
:108E100007015651146E156AFF0E141801E1155022
:108E20000FE05651562B19080BE155811200020E26
:108E30000701565D04E3190E565D01E25581566B3C
:108E4000120030D800090FE007015751146E156A5F
:108E5000FF0E141801E115500FE05751572B190858
:108E60000BE155831200020E0701575D04E3190E52
:108E7000575D01E25585576B12001BD8010A04E0CB
:108E8000030A02E0010A01E1010C000C12D80408F7
:108E900001E1000C010C0DD8010A02E0020A01E117
:108EA000010C000C06D8020A02E0010A01E1010CE3
:108EB000000C0601100EB95D0E0EBA5901E3000C4C
:108EC000B80EB95D0B0EBA5901E3020C340EB95D50
:108ED000080EBA5901E3010CE80EB95D030EBA5948
:0C8EE00001E3030C040C91DF21EF47F0CC
:048EEC009050080B8F
:108EF00001E1010C020C60D8FE0EDB0404E0FE0E62
:108F0000DB50020802E1010E01D0000E5AD054D805
:108F1000AAEC2DF0FE0EDBCFE6FF69EC38F0E5524F
:108F2000FD0EDBCFE6FFFE0EDBCFE6FF09D8E552F4
:108F3000E552FE0EDBCFE6FF6CEC38F0E55241D097
:108F40003BD8AAEC2DF0410E2ED84E0E2CD8FD0E9B
:108F5000DB50300928D835D02FD8C8DF146EFE0E6C
:108F6000DB50145C11E00601D8510601425D060198
:108F7000D9510601435902E2010E14D0FE0EDB5016
:108F8000020A06E0030A02E0000E0CD0909601D01F
:108F90009086205006E0AADFE66EE66AB8DFE5526A
:108FA000E552010E0ED0E66EFE0EDBCFE6FF23EC9F
:108FB00038F0E552E5521200D9CFE6FFE1CFD9FFF4
:0A8FC0001200E552E7CFD9FF1200BE
:068FCA0007014CAB010C95
:108FD0008FA6010C000C4DD8AAEC2DF0FE0EDBCFB5
:108FE000E6FF69EC38F0E5528F50080B01E0010E06
:108FF000E66EFE0EDBCFE6FF09D8E552E552FE0E27
:10900000DBCFE6FF6CEC38F0E55238D032D8420EB8
:1090100027D8590E25D807014C51200B03E0FD0E2F
:10902000DB5002E1420E01D04E0E1AD827D021D8D3
:109030008F50080B01E0010E146EFE0EDB50145C25
:1090400002E1000E0CD0FE0EDB50E8B08F86E8A0E7
:109050008F96205003E0E66ABEDFE552010E0ED087
:10906000E66EFE0EDBCFE6FF23EC38F0E552E5526C
:109070001200D9CFE6FFE1CFD9FF1200E552E7CFCA
:04908000D9FF120002
:0C9084009150400B01E0010C000C47D89B
:10909000AAEC2DF0FE0EDBCFE6FF69EC38F0E552CE
:1090A000FD0EDBCFE6FFFE0EDBCFE6FF09D8E55273
:1090B000E552FE0EDBCFE6FF6CEC38F0E55234D023
:1090C0002ED8530E23D8490E21D8FD0EDB5002E1D5
:1090D000410E01D0540E1AD827D021D8D3DF146EF8
:1090E000FE0EDB50145C02E1000E0FD0FE0EDB041E
:1090F00002E1918C01D0919C205006E0C3DFE66E26
:10910000E66AC5DFE552E552010E0ED0E66EFE0EB0
:10911000DBCFE6FF23EC38F0E552E5521200D9CF61
:10912000E6FFE1CFD9FF1200E552E7CFD9FF1200E9
:10913000D9CFE6FFE1CFD9FFE150FD0FE96EFF0E79
:10914000DA20EA6EEE50ED100FE041EC1CF0E5C5C0
:10915000E6FFFD0EDBCFE6FFFE0EDBCFE6FF53ECB6
:1091600018F0E552E552E552E552E7CFD9FF12007B
:10917000D9CFE6FFE1CFD9FFE6520F011451151107
:109180001FE023D866EC1DF0E552E552DF6E0701C3
:109190003651DF5C11E020A613D0DFCFE6FFE66A90
:1091A00014D8720EE66E1F0EE66E1CEC2DF0146ED7
:1091B000060EE15E145004D008D8BADFE552E5523D
:1091C000E552E552E7CFD9FF120014CFE6FF15CFE5
:0491D000E6FF1200A4
:0C91D400CAEC37F000094CE0B7EC37F0B3
:1091E0000001F86F6151EA6A620FE96E000EEA222F
:1091F000F8C0EFFF960E615D01E2612B3B0EF85D5A
:10920000E9E162515E0A07E0650A1EE13B0EE66E87
:1092100050EC38F017D0050E606F61C0E6FF620EAB
:10922000E66E000EE66E23EC4AF0E552E552E5529A
:10923000620EE66E000EE66E010EE66E8AEC20F01F
:10924000E552E552E55213D0616B6151612BEA6A38
:10925000620FE96E000EEA22EFCFF8F0F8C0E6FFE9
:1092600038EC38F0E5523B0E0001F85DEEE100010C
:06927000616BB0D7120093
:0A927600200EF66E080EF76E000ED3
:10928000F86E07010900F550166F0900F550176FC9
:1092900003E1166701D03DD00900F550116F0900B8
:1092A000F550126F0900F550136F09000900F550D1
:1092B000E96E0900F550EA6E090009000900F55051
:1092C000146F0900F550156F09000900F6CF18F763
:1092D000F7CF19F7F8CF1AF711C7F6FF12C7F7FF44
:1092E00013C7F8FF0701145302E1155307E0090003
:1092F000F550EE6E1407F8E21507F9D718C7F6FF18
:1093000019C7F7FF1AC7F8FF07011607000E175B0A
:04931000BFD71200B1
:0C93140039D84EC7E6FF4FC7E6FF44D82B
:1093200003D8E552E55227D038D8570E13D8FC0E93
:10933000DBCFE6FFFD0EDBCFE6FF13D025D834D818
:1093400001D819D02AD8420E05D850C7E6FF51C718
:10935000E6FF07D0E66E28D823EC38F0E552E55258
:10936000120022D844EC35F0E552E552E552E552C0
:10937000E7CFD9FF1200E55217D86CEC38F0E55270
:10938000E552E7CFD9FF1200D9CFE6FFE1CFD9FFF1
:109390000BD869EC38F0E5521200D9CFE6FFE1CFE7
:1093A000D9FF530EAAEF49F0FE0EDBCFE6FF120005
:1093B000420E44D8450E42D8530E40D8540E3ED8E3
:1093C00078EC38F0FAC6E6FFFBC6E6FFE66A94ECF6
:1093D00049F0E552E552E552120078EC38F0F7C654
:1093E000E6FFE66A60EC48F0E552E55278EC38F0CA
:1093F000F8C6E6FFE66A55EC43F0E552E55278EC34
:1094000038F0F9C6E6FFE66ACFEC42F0E552E552E5
:10941000E66A6CEC38F0E5521200AAEC2DF0470E2B
:109420000DD8C6DFEDEF49F0AAEC2DF0530E06D8AB
:10943000BFDFE66A6CEC38F0E5521200E66E38ECFD
:0694400038F0E5521200B5
:0A944600D9CFE6FFE1CFD9FFFC0EFD
:10945000DBCFF3FFDB06F350000915E038D8EFCF80
:1094600014F0610E145C09E332D8EF507A0805E37A
:10947000200E146E2CD81450EF5EFD0EDB2AFE0E6B
:10948000E6E3DB2AE4D7E552E7CFD9FF1200D9CFD4
:10949000E6FFE1CFD9FF610EF36EFE0EDBCFF4FFE6
:1094A000F350F45C0EE3FE0EDB507A080AE3200E64
:1094B000146EFE0EDBCFE7FF1450E75EFE0EE7CF23
:1094C000DBFFFE0EDB50E552E7CFD9FF1200FD0EA9
:0C94D000DBCFE9FFFE0EDBCFEAFF12004D
:0494DC00D9CFE6FFFF
:1094E000E1CFD9FF030EE126FC0EDB50E76E34D846
:1094F000E7501426000E152214C0DEFF15C0DDFF54
:10950000020EDB6A29D8DECF16F0DDCF17F0165039
:10951000145C1750155812E2FD0EDBCFE9FFDB2A71
:10952000FE0EDBCFEAFF01E3DB2A020EDBCFE7FF13
:10953000EF50E726020EE7CFDBFFE4D7020EDB5049
:10954000146E030EE15C02E2E16AE552E16E145032
:10955000E552E7CFD9FF1200FD0EDBCF14F0FE0E6F
:06956000DBCF15F0120044
:0A95660033D8AAEC2DF0FE0EDBCF87
:10957000E6FF69EC38F025D80AD8E552E552E55205
:10958000FE0EDBCFE6FF6CEC38F0E55225D01FD89D
:10959000460EE66EFE0EDBCFE6FF23EC38F0E5521A
:1095A00010D862EC35F0E552E552E55215D00FD8EF
:1095B000205006E015D8E66AD6DFE552E552E552BE
:1095C0000BD0E552FC0EDBCFE6FFF0EF4AF0D9CF2F
:1095D000E6FFE1CFD9FF1200E552E7CFD9FF120035
:0E95E000FD0EDBCFE6FFFE0EDBCFE6FF120036
:0295EE00D76A3A
:1095F000D66AA10ED56E12006CC6E6FF6DC6E6FFF8
:1096000015D8E552E552000905E106016B0E6C6FB5
:10961000F00E6D6F070ECD6E9E909F809D806DC683
:1096200014F01450CF6E6CC6CEFF1200D9CFE6FFF7
:10963000E1CFD9FFFD0EDBCF14F0FE0EDBCF15F02E
:10964000770E145CEE0E15580CE3D950FD0FE96E41
:10965000FF0EDA20EA6E5F0ED880EE54F20EED5463
:1096600002E2000E01D0010EE552E7CFD9FF120051
:1096700006500B02F3CF02F0F4CF03F00C02F350CC
:109680000326000EF420046E06500D02F35004264B
:10969000000EF420056E06500E02F350052607500A
:1096A0000B02F3500326F4500422000E052207504B
:1096B0000C02F3500426F450052207500D02F3501B
:1096C000052608500B02F3500426F45005220850DA
:1096D0000C02F350052609500B02F3500526120028
:1096E0000F01E40E196F550E7E6EAA0E7E6E5F8B13
:1096F000188BFD0E186F5F9B1769166912000F011A
:109700005F0E256F020E246F400E236F896A8A6AEE
:109710008B6A8C6E100E8D6E8E6A8F6A300E906E14
:10972000916A3F0E926E936AB80E946E956A966A2D
:10973000120E976E240E986E220E996E9A6A12007F
:10974000EC010433030A0004099A0507330705CD29
:109750000803660A01CD0C00FFFF0F29000F7C00F3
:1097600000CE0001210103740104C601051902069F
:109770006B0207BE020810030963030AFFFF0F6CA8
:1097800007A60EF714EE1B8D275F37C646E9526C0D
:0597900061B27020CB66
:0197950010C3
:0A979600056A046A036A026A200EE5
:1097A000E76ED89006360736083609360236033695
:1097B000043605360B50025C0C5003580D5004580B
:1097C0000E50055809E30B50025E0C50035A0D5021
:0E97D000045A0E50055A062AE72EE4D712005E
:0297DE00FE0E7D
:1097E000E3CFE9FFFF0EE3CFEAFFE9CFF3FFEACFD4
:1097F000F4FFFB0EE35003E1FC0EE35009E0FB0E27
:10980000E30602E2FC0EE306FD0EE350EE6EF1D736
:02981000120044
:0E9812000803C803D003D303E003E603E60314
:10982000E503DB03DD035D032E07D106CB06B70698
:0E983000B506C506A106900698069006CD0660
:02983E00056AB9
:10984000046A100EE76ED8900836093604360536DD
:109850000D50045C0E50055805E30D50045E0E508B
:0A986000055A082AE72EF0D712007F
:06986A001EEE00F02EEEE0
:1098700000F0F86A019C55EC4CF03BEC49F0A5EC8B
:0A98800036F0E3EC36F0FBD71200DF
:06988A00FF0EE350246E06
:10989000480E01D04C0EE76EE72EFED7E76AE72EA2
:0A98A000FED7242EF7D700001200B7
:0698AA00160EF36E00EE45
:1098B00000F00F0E01D81200EA6002D0EE6AFCD769
:0A98C000F350E9601200EE6AFCD7D5
:0698CA00056A080EE76EBE
:1098D000D890093605360E50055C02E3056E092A5C
:0698E000E72EF7D712008D
:0A98E60000008403460508078C0A01
:0C98F0003C0FEC134416F41A781E4821BB
:0498FC004849524144
:089900004B453B0035303B00F4
:049908000400120045
:04990C000A000A0043
:1099100096004B004B009600C800C8006400C800C9
:10992000960078006E000A141414141414141464AD
:10993000C8B80B941170172823C8326842384AD827
:079940005990657094FFFFD0
:03994700FFFFFF20
:01994A000F0D
:01994B004ECD
:04994C00C4095834BE
:02995000FA001B
:020000040030CA
:0100000015EA
:0100010002FC
:0100020056A7
:0100030026D6
:01000400F902
:010005008179
:010006008178
:01000800FFF8
:01000900C036
:01000A00FFF6
:01000B008074
:01000C00FFF4
:01000D0040B2
:00000001FF
